:020000040800F2
:10000000203C00208D010008E5430008454400081D
:10001000090100080B0100080000000000000000BA
:100020000000000000000000000000000F010008B8
:1000300011010008000000001301000835560008F7
:1000400000000000000000000000000000000000B0
:1000500000000000000000000000000000000000A0
:100060000000000000000000000000000000000090
:100070000000000000000000000000000000000080
:100080000000000000000000000000000000000070
:100090000000000000000000000000000000000060
:1000A0000000000000000000000000000000000050
:1000B0000000000000000000000000000000000040
:1000C0000000000000000000000000000000000030
:1000D0000000000000000000000000000000000020
:1000E0000000000000000000000000000000000010
:1000F0000000000000000000000000000000000000
:1001000040380008FEE7FEE7FEE7FEE7FEE7FEE711
:10011000FEE7FEE7FEE72020174D01202968014396
:100120002960361F37602F4600B500BF3D680220AA
:100130000540FBD01120114908601148786000206B
:10014000F862104839680143396000BF3D680E48C5
:100150000540FBD03D1D0C3E032131600221716042
:10016000B7602F4601F0FEFB7D680C200540082D8E
:10017000FAD180CE00BD01BC001002400020024038
:1001800000801004000000010000000200B500BF64
:10019000104D85F30888104D85F30988022585F3F5
:1001A0001488BFF36F8F0D4E0D4DAB460D490E48B1
:1001B0000D6805430D600D490D480D6885430D60C0
:1001C000FFF7AAFF0B48056801200543A847DFE7B2
:1001D00000BD0000203C0020203E0020043F002005
:1001E000103F00201410024014007E00281002402E
:1001F00000007E0000010008043F0020203E002097
:1002000000000000000000000000000000000000EE
:100210000A0000000000000000C0000800C0000844
:10022000B80000204C000020C093442300000000D0
:10023000C3414E4431680F40361D70470000000036
:10024000C24F522031680F43361D70470000000036
:10025000C3584F5231684F40361D704700000000B0
:10026000C6494E5645525420FF43704700000000D7
:10027000C2303D20002F01D0002701E001277F423E
:100280007047000000000000C3303C3E002F01D149
:10029000002701E001277F4270470000700200083C
:1002A000C2303C20002F01D4002701E001277F420B
:1002B00070470000A0020008C2303E20002F01DC81
:1002C000002701E001277F42704700000000000086
:1002D000C13D20203068874201D0002701E001277E
:1002E0007F42361D70470000D0020008C23C3E200D
:1002F0003068874201D1002701E001277F42361D87
:100300007047000000000000C13C20203068874298
:1003100001DC002701E001277F42361D7047000005
:1003200060020008C13E20203068874201DB0027C0
:1003300001E001277F42361D70470000EC020008F3
:10034000C23C3D203068874201DA002701E00127E6
:100350007F42361D7047000000000000C23E3D2075
:100360003068874201DD002701E001277F42361D0A
:100370007047000000000000C2553E2030688742F0
:1003800001D3002701E001277F42361D704700009E
:1003900078030008C2553C203068874201D8002706
:1003A00001E001277F42361D7047000094030008DA
:1003B000C344303C002F01D4002701E001277F42D5
:1003C000361D7047B0030008C344303D31680F4309
:1003D000002F01D0002701E001277F42361D704722
:1003E00000000000C2443D2007CE3B1C0027801ABD
:1003F0008B41384300D1FF43704700005C03000885
:10040000C34D494E01CE874200DD074670470000CC
:1004100000040008C34D415801CE874200DA074668
:100420007047000008030008C657495448494E2049
:1004300030683F1A716830680D1AAF4201D8002742
:1004400001E001277F42083670470000B80200082B
:10045000C64C534849465420384680CE87407047A2
:1004600000000000C652534849465420384680CE0A
:10047000C740704764040008C74152534849465476
:10048000384680CE0741704700000000C7455845F8
:10049000435554450120384380CE00470121704622
:1004A0008843026810470000391C80CEF6D07046A1
:1004B000001D004701CEB842F0D180CEF7E7000022
:1004C0000099491C0091E9D703B0F0E70099C919D8
:1004D000009180CEE2D703B0E9E7000002CE01240C
:1004E000E40773465B1E1A680919781A07B480CEB0
:1004F000DDE7000002CEB942F1D180CECEE70000A8
:1005000040020008C54C45415645202002B000BDC0
:1005100000000000C63F4C45415645203F1C80CEA0
:1005200000D1704702B000BD00000000C14920208A
:10053000361F3760009F01983F187047500200082F
:10054000C14A2020361F3760039F04983F18704728
:1005500040050008C6554E4C4F4F502003B0704721
:10056000E4030008C3533E44FD17361F37602F468F
:100570007047000050040008C44E4F4F5020202008
:100580007047000024030008C24D2B2003CEFA1749
:10059000C91950410746361F31607047880200086C
:1005A000C2312B207F1C7047A0050008C2312D20CE
:1005B0007F1E70478C040008C12B20203068361D38
:1005C0003F18704740030008C12D20203068361DB9
:1005D000C71B704730020008C64E454741544520AE
:1005E0007F42704764050008C2442B2007CE801864
:1005F0004F41361F30607047E8050008C2442D2087
:1006000007CE101AB9410F46361F30607047000000
:1006100054050008C7444E45474154453068002101
:100620004042B9410F46306070470000FC050008A9
:10063000C73F4E45474154453F1C80CE00D57F42C1
:1006400070470000D8050008C3414253002F00D571
:100650007F42704778040008C44441425320202060
:100660003F1CDBD470470000C8030008C344322A93
:10067000306800187F413060704700006C06000849
:10068000C344322F306840107F108941C9070843A6
:100690003060704714060008C12A202031684F439B
:1006A000361D704758060008C3554D2A3846316834
:1006B00040B40A04120C0B0C0404240C050C16465E
:1006C00066431F466F4318466043010C000436180A
:1006D0004F4128465043010C000436184F4135461F
:1006E00040BC35607047000088050008C24D2A20D4
:1006F00035687D4000B520B4002F00D57F423568B5
:10070000002D00D56D423560FFF7D0FF20BC002DD5
:1007100001D5FFF783FF00BD98060008C6554D2F91
:100720004D4F442001CE3168202400224918404119
:1007300013465341C01B5B4101D0491C00E0C01966
:10074000641EF3D10F46306070470000B805000802
:10075000C6464D2F4D4F442000B580B435687D40CE
:1007600020B480B480CEFFF77BFF009D002D00D524
:100770006D42361F37602F46FFF7D4FF15480740FC
:1007800020BC002D01D4002501E001256D42002D83
:10079000EFF3008001B430683760074601BC80F396
:1007A000008800D57F4220BC002DEFF3008001B40B
:1007B00030683760074601BC80F3008808D57F4267
:1007C0003068002804D07F1E009D30682D1A3560E7
:1007D00001B000BDFFFFFF7F00000000C6534D2F9A
:1007E00052454D2000B5306801B480B480CEFFF78B
:1007F00037FF009D002D00D56D42361F37602F4614
:10080000FFF790FF20BC009C6C40002C00D57F427D
:1008100020BC002DEFF3008001B43068376007463C
:1008200001BC80F3008800D57F42306837600746FE
:1008300000BD0000AC050008C42F4D4F442020200F
:1008400000B580B43168CF1720BC361F37602F4603
:10085000FFF7C8FF00BD000014040008C12F2020CE
:1008600000B580B43168CF1720BC361F37602F46E3
:10087000FFF7B8FF361D00BD80060008C2552F20C7
:10088000361F0021316000B5FFF74CFF361D00BD5B
:100890005C080008C34D4F4400B5FFF7D1FF80CE80
:1008A00000BD0000EC060008C24D2F2000B5FFF788
:1008B00099FF361D00BD000038080008C64D552FB1
:1008C0004D4F442000B580B4009F361F0021316099
:1008D000FFF728FF20BC80B42F46FFF723FF20BC82
:1008E000361F37602F4600BDA8080008C52A2F4DC7
:1008F0004F44202000B580B480CEFFF7F9FE20BC25
:10090000361F37602F46FFF76DFF00BD5007000808
:10091000C22A2F2000B5FFF7EDFF361D00BD0000F5
:1009200004050008C34E4950361D7047A80600084C
:10093000C45455434B202020361F716831607760C6
:100940007047000048060008C45049434B2020204F
:10095000BF00F7597047000030060008C4524F4CE2
:100960004C202020B800002801DC80CE704737588A
:10097000011F72583250081CFAD1361D7047000012
:1009800014050008C3524F543D46776831687160C2
:100990003560704724090008C42D524F5420202090
:1009A0003D4637687168316075607047940800088B
:1009B000C23E522080B480CE704700004809000833
:1009C000C2523E20361F376080BC7047C009000805
:1009D000C2524020361F3760009F704784090008CC
:1009E000C3323E5203CE01B480B40F1C70470000E6
:1009F000E0090008C332523E03BC083E3160776014
:100A000007467047F4090008C33252400098019924
:100A1000083E316077600746704700007C08000898
:100A2000C453574150202020306837600746704734
:100A3000200A0008C3445550361F37607047000035
:100A4000BC080008C44F564552202020361F37608E
:100A50007768704730090008C444524F5020202066
:100A600080CE7047340A0008C53244524F502020CF
:100A70007768083670470000680A0008C532535787
:100A800041502020706877600746B0683168B160D7
:100A9000306070475C090008C43244555020202063
:100AA000083EB16831607760704700007C0A00083A
:100AB000C5324F5645522020083E3169316077607B
:100AC000F7687047440A0008C43F4455502020206E
:100AD000002F01D0361F376070470000980A0008C9
:100AE000C3535040361F376037467047E00A00084E
:100AF000C35350213E4680CE70470000080A0008CC
:100B0000C3525040361F37606F467047000B0008D5
:100B1000C3525021BD4680CE70470000580A0008DD
:100B2000C5434F554E5420207D1C3F78361F3560FD
:100B300070470000F00A0008C72F535452494E472F
:100B40003168CD1B70683F1877602F46361D70479F
:100B5000B00A0008C4534B495020202003CE401C4B
:100B6000401E04D00A78BA4201D1491CF8E7361F6A
:100B70003160074670470000540B0008C4534341DE
:100B80004E20202003CE401C401E04D00A78BA42DA
:100B900001D0491CF8E7361F316007467047000056
:100BA000100B0008C2533D2003CE3F1C07D0027833
:100BB0000B78401C491C9A4201D17F1EF7D102D10B
:100BC00001277F4200E00027704700002C05000845
:100BD000C7434F4D504152457168CD1B00B520B4FD
:100BE00071688F4200DB0F1C31687160361D00BFD9
:100BF000002F23D075682D78346824782C1B002CA6
:100C0000EFF3008001B4361F71683160B168716024
:100C1000B760274601BC80F3008804D001B080B4DF
:100C20000027361D09E037687F1C75686D1CB068A9
:100C3000441E7760B5602746361DD9E780BC002F7B
:100C4000EFF3008001B4083601BC80F3008807D0C0
:100C5000002F01D4002701E001277F420120074334
:100C600000BD202000B5B16802B4716802B43168DB
:100C700002B480B480B0484601B4E946F768103643
:100C80004D462D694C46E4684B465B68E31A5B1C95
:100C90005B19083E336077602F4600BFFFF72AFCE0
:100CA0000F0D0008009D019805442D784C46A4685E
:100CB0002478AC4226D1009D019805444C46A46896
:100CC0004B465B680C3E34607560B7601F46FFF7AB
:100CD0006BFF002F80CE15D0009D019805444C4637
:100CE000E468009B019803444A4612699A1AA21AC2
:100CF00003B00C3E32607560B7600B4F01BC81469B
:100D000004B000BD0098401C0090CBD703B04D4606
:100D10002D694C46E4680C3E34607560B76000276E
:100D200001BC814604B000BDFFFFFFFFDC070008E7
:100D3000C6534541524348207068874200B502DDE2
:100D40000027361D00BD002F02DC064F361D00BDFA
:100D50007068002802DC0027361D00BDFFF782FF07
:100D600000BD0000FFFFFFFF200B0008C5434D4FF3
:100D7000564520203B1C83CE00D17047021C0A43FD
:100D80001A430324144006D10A680260091D001D9D
:100D90001B1FF9D170470A780270491C401C5B1E6A
:100DA000F9D17047300D0008C6434D4F56453E20DF
:100DB0003B1C83CE00D17047C018C918021C0A43DF
:100DC0001A430324144006D1091F001F0A68026059
:100DD0001B1FF9D17047491E401E0A7802705B1E26
:100DE000F9D170476C0D0008C3555043612F00B511
:100DF00003DB7A2F01DCDF20074000BDD00B0008A9
:100E0000C55550504552202030683F183068376033
:100E1000074600B5FFF76EFB430E0008009D0198E2
:100E200005442D78361F37602F46FFF7DFFF009D02
:100E3000019805442F7080CE0098401C0090EDD79B
:100E400003B000BDA40B0008C5504C414345202011
:100E500000B5306801B480B47F1C30683760074645
:100E600001F05CFF20BC10BC2C7000BD980900088C
:100E7000C24F4E2001204042386080CE70470000B3
:100E800078050008C34F46460020386080CE704782
:100E9000D0090008C232402003CF361F0746316018
:100EA00070470000940E0008C23221203A1C83CE05
:100EB00003C27047000E0008C446494C4C20202055
:100EC0003A1C83CE002803D00A70491C401EFBD177
:100ED0007047000028040008C22B212030683968C0
:100EE000091839607768083670470000D80E000886
:100EF000C4494E43522020203868401C386080CEC0
:100F000070470000E80D0008C444454352202020EB
:100F10003868401E386080CE70470000700E0008B0
:100F2000C14020203F687047A80D0008C2574020EC
:100F30003F887047480E0008C24340203F78704702
:100F4000840E0008C1212020306838607768083698
:100F5000704700002C0F0008C257212030683880ED
:100F60007768083670470000380F0008C243212018
:100F7000306838707768083670470000100900083C
:100F8000C8544553542D4249542020203F7831689D
:100F90000F40361D70470000B80E0008C753455477
:100FA0002D424954306839780143397077680836E2
:100FB000704700001C070008C952455345542D4294
:100FC0004954202030683978814339707768083671
:100FD00070470000C80A0008C54E414D453E20201C
:100FE0003D781F200540ED192D1D2F4603218F430D
:100FF00070470000D80F0008C53E4E414D452020E7
:1010000000B500BF3F1F3D6880200540FAD000BDFD
:1010100000B500BF3F68002F2BD03D781F20054052
:101020003068854223D17D1C0C3E3169316075608A
:10103000B760F768FFF7B8FD002F80CE17D0776054
:10104000361DFFF7CDFF35682D7840200540EFF3C2
:10105000008001B4361D01BC80F3008803D0361F28
:101060003760054F02E0361F3760012700BD3F1F84
:10107000D0E70027083600BDFFFFFFFF002F00B5B7
:1010800001D108360CE075682D7830682D183C6861
:10109000641E2C40641CA400E4192746FFF7B8FF27
:1010A00000BD000001CE30380BD40A2802DBC01F7F
:1010B0000A2806DBB84204DA01277F42361F306077
:1010C00070470027704700003F1D7047BF00704702
:1010D0003F1F7047361F3760042770473D0C361F8F
:1010E00037602F4600B501F013F801F011F800BD8C
:1010F00031680D0C083E3560776000B500F02EFDBC
:10110000BF1C00F02BFD00BD30680740002F01D050
:10111000002701E001277F423068002801D4002524
:1011200001E001256D427D402F46361D704720208D
:101130003F1D3168CF1B7F10154D3D40FC0A1548FF
:10114000044024042C43083E37607460B760124F9B
:1011500000B5FFF7D9FF1148074031680F43361F2C
:10116000B168316077600E4FFFF7CEFF0D48074042
:1011700031680F437068002801D4002501E0012583
:101180006D42094805403D432F46083600BD00002A
:10119000FF070000FF030000000020000020000007
:1011A00000004000000800000000000400B5FFF748
:1011B000BFFF0148074300BD00D000F0361F376075
:1011C000024F00B500F0A4FF00BD000000B5000014
:1011D000361F3760024F00B500F09AFF00BD0000D7
:1011E00000BF0000361F71683160776000B5FFF7FF
:1011F000DDFF306837600746FFF77AFF00BD20202B
:10120000361F3760044F00B500F082FF361F37608D
:10121000024F00F07DFF00BD361F00003760000068
:10122000361F3760074F00B500F072FF361F37607A
:10123000054F00F06DFF361F3760044F00F068FF68
:1012400000BD000070460000401E0000076800005E
:1012500000B500F0BBFEFFF7A9FFFFF73FFF00BDA1
:1012600000B500F0B3FE0220074080CE01D0FFF7AA
:10127000AFFFFFF7EDFF00BD00B5FFF79FFF00BD1B
:10128000361F37607046401E0768401D004700004B
:10129000361F3760009F7F1E3978C919091D032248
:1012A0009143491C00917047080F0008C7414C4901
:1012B000474E4544FF1C03218F437047361F37605C
:1012C0007046401E076800BDB80F0008C8434F4D68
:1012D00050494C452C20202000B5FFF7B9FF00BD38
:1012E000F80F0008C53E424F44592020BF687047A0
:1012F00000B5FFF76DFFFFF761FF361F3760024F44
:10130000FFF7A6FF00BD0000BC12000800B5FFF704
:101310005FFFFFF753FF361F3760042700F072FEB0
:1013200000BD202000B500F0ABFE00F07FFFFFF70E
:10133000EDFF30683760074600F0DAFE00F0ACFEE3
:1013400000BD202000B520BC01218D43361F376031
:101350002F4600F0F9FEFFF743FE3F1DFFF742FF67
:1013600000BD000000B500BF00F0D8F8000000206C
:10137000800F0008C3494D4D0249012040420860DA
:101380007047000000000020CC120008813A2020A5
:1013900000B501F03FFD01F009FD00F047FF00F04E
:1013A000DBFE01F043FFFFF767FF00BD200F0008E1
:1013B000C73A4E4F4E414D4500B501F0F7FC00F0E5
:1013C00089FE00F003FE00F06BFD306838600027F6
:1013D000361D00F08DFE00F0F9FD01F027FFFFF74C
:1013E0004BFF00BD580F000885444F45533E202059
:1013F00000B500F0B1FD00F0DFFF05444F45533E5E
:10140000361F37600C4FFFF767FF00F0A5FD00F0B7
:10141000D3FF0161FFF7F4FE00F09EFD00F0CCFF6A
:1014200001620000FFF7FCFE00F096FD00F0C4FF33
:101430000163000000BD000044130008E813000829
:10144000C64352454154452000B500F02BFE00F044
:1014500017FE30683760074600F0E8FEFFF748FFE8
:1014600000F06EFF00F018FE00BD0000E41200085E
:10147000C73C4255494C445300B500F013FE00F000
:10148000FFFD30683760074600F0D0FEFFF73EFFF3
:1014900000F056FF00F000FE00BD00008C130008B5
:1014A000C8434F4E5354414E5420202000B5FFF7FF
:1014B00039FFFFF747FF361F37607046401E076849
:1014C00000BD0000A0140008C932434F4E535441E0
:1014D0004E54202000B5FFF725FF00F009FEFFF76E
:1014E00031FF083E77607046401E076841683160F2
:1014F00000BD0000C8050008C85641524941424C91
:101500004520202000B500F08DFDFFF70BFF361FB2
:101510003760042700F094FDFFF714FF361F376093
:101520007046401E076800BD40140008C74255467B
:101530004645523A00B500F075FDFFF7B7FF00F0E1
:101540007FFD00BD2C150008C455534552202020B6
:1015500000B5FFF7E7FEFFF7F5FE361F3760704670
:10156000401E07685F4400BD704700004815000832
:10157000C54445464552202000B500F053FDFFF715
:10158000D1FE361F3760042700F05AFDFFF7DAFE60
:101590007046401E006801680122114308BC9E4647
:1015A0000847000000B500BFFFF7B8FF04000020A7
:1015B00000B500F05DFC3F68002F80CE05D080CEE6
:1015C000FFF74EFE00F094FD05E03D4677680836D3
:1015D00001200543A84700BD00B500F0BDFC00F0A8
:1015E000EBFE1E496E76616C6964206F70657261F6
:1015F000746F7220666F72207468697320747970DA
:1016000065000000361F3760014F00F007FF00BD86
:10161000F3FFFFFF7146491E0868491D8E460760AB
:1016200080CE7047361F37607146491E0868491DD5
:101630008E46076870470000C8140008C556414C24
:101640005545202000B5FFF797FE80B480CE00F00E
:10165000E9FCFFF767FE20BC361F37602F4600F01D
:10166000E1FC306838600427361D00F0E9FCFFF724
:1016700069FE361F37607046401E076811480568CE
:10168000104900200860002DEFF3008001B4361FE0
:1016900037602F4601BC80F3008806D1361F0A4F01
:1016A0000A493160FFF784FF0BE0012F06D1361F96
:1016B000074F08493160FFF77BFF02E0FFF78CFF1F
:1016C00080CE00BD04000020240F0008241600086E
:1016D000480F000814160008380B000882544F20E9
:1016E0000120014908607047040000206C0F0008C9
:1016F000C55041555345202000B500BFFFF748FFB6
:101700000800002000B500F061FC361F3760042798
:1017100000F078FC00BD202000B500F057FC01204F
:10172000074330683760074600F02CFA00BD2020E0
:1017300000B500F04BFC00BD0120074300B500F0F0
:10174000D7FC00BD361F3760034F00B5FFF788FD9B
:10175000FFF7F2FF00BD00009C040008361F376051
:10176000034F00B5FFF77CFDFFF7E6FF00BD00006B
:10177000A8040008361F3760034F00B5FFF770FD5F
:10178000FFF7C0FF00BD00009C040008361F376053
:10179000034F00B5FFF764FDFFF7B4FF00BD000085
:1017A000A8040008361F3760034F00B5FFF758FD47
:1017B00000F09EFC00BD000080120008361F37605C
:1017C000024F00B5FFF788FD00BD0000600A000869
:1017D000361F3760024F00B500F09AFC00BD0000D4
:1017E00000BD0000361F3760044F00B5FFF738FD1D
:1017F000FFF788FFFFF79CFF00BD0000DC04000836
:10180000361F3760044F00B5FFF72AFDFFF77AFF58
:10181000FFF78EFF00BD0000F4040008361F37609C
:10182000044F00B5FFF71CFDFFF786FFFFF774FFBD
:1018300000BD0000C0040008361F3760044F00B52B
:10184000FFF70EFDFFF778FFFFF766FF00BD000012
:10185000CC04000800B500BFFFF760FE0C000020BC
:1018600005480568361F37602F4600B5FFF760FF53
:1018700001490F6080CE00BD0C000020361F37608C
:10188000034F00B5FFF7ECFCFFF73CFF00BD000085
:10189000B404000800B5FFF76DFF306837600746F5
:1018A000FFF73AFF00BD202000B500BF361F3760AC
:1018B000374600F0CDFA3F6830688742EFF300808A
:1018C00001B47768083601BC80F3008802D0FFF7C6
:1018D00023FFEBE700BD202000B5FFF76FFFFFF708
:1018E000E3FF02490F6080CE00BD00000C00002025
:1018F00000B5FFF763FF06480568361F37602F46BF
:10190000FFF720FFFFF7D0FF01490F6080CE00BD39
:101910000C00002000B5FFF739FF00BDDC16000801
:10192000C244492072B670477C0B0008C24549206A
:1019300062B67047F00E0008C25B4920EFF31080DA
:1019400072B601B4704700003C160008C2495D2021
:1019500001BC80F3108870479C0F0008C7534554A2
:101960004D41534B3D683068C4432C40706804437C
:101970003C60B7680C367047B0090008C7494E494B
:10198000542D494F00B500BF3D68002D04D03D687F
:101990007C682C600837F7E780CE00BD07480568F3
:1019A0008020054000B508D0054D0648686006480F
:1019B0006860802029698143296100BD10200240B0
:1019C0000020024023016745AB89EFCD083E134953
:1019D00031607760124F00B53068451E002DEFF37F
:1019E000008001B4356001BC80F3008804D0FD683C
:1019F00001200540002DEFD1FD6834242C40FC600F
:101A000030680028EFF3008001B42F46361D01BC7A
:101A100080F3008801D10348074300BD0000100097
:101A2000002002400000008000B5FFF7B7FF084922
:101A300001200D6805430D603068388077680836EE
:101A4000FFF7C4FF024901200D6885430D6000BD0A
:101A5000102002400B483F1A00B5FFF79FFF0A4DC8
:101A600002202969014329616F61402029690143EE
:101A7000296180CEFFF7AAFF044902200D68854343
:101A80000D6000BD00000008002002401020024050
:101A900000B5FFF7C9FF80CE00BD20203D7830683B
:101AA000854200B502D17768083600BD3D46012168
:101AB0008D4301200740EFF3008001B42F4601BCA5
:101AC00080F3008806D031680D023C782C433760E3
:101AD000274605E07D782D0231680D4337602F469B
:101AE000306837600746FFF7D3FF00BD074D316808
:101AF0000D40083E3560776000B5FFF7C9FF3168DB
:101B00000D0CBF1C3560FFF7C3FF00BDFFFF0000D9
:101B1000083E044931607760034F00B5FEF788FC4A
:101B200000BD000000000008000010082019000897
:101B3000C3432146361F376000B5FFF7E9FF002F8A
:101B400080CE02D0FFF7AAFF03E0306838707768D4
:101B5000083600BD5C190008C3572146361F3760A0
:101B600000B5FFF7D5FF002F80CE02D0FFF790FF22
:101B700003E0306838807768083600BD70140008CC
:101B8000C2214620361F376000B5FFF7C1FF002F86
:101B900080CE02D0FFF7AAFF03E030683860776894
:101BA000083600BD38190008C7464C455241534518
:101BB00030683F1830683760074600B5FEF79AFC7A
:101BC0000B1C0008009D01980544361F37602F4606
:101BD000FFF79EFF002F80CE09D0009D019805449D
:101BE000361F37602F46FFF735FF084F07E0009D8F
:101BF0000198054406482860361F3760042700987E
:101C0000C019009080CEDDD703B000BD00080000F1
:101C1000FFFFFFFF083EB1683160776000B5FFF756
:101C2000C7FF31687D1811480468083E346077604A
:101C30002F46FFF7A7FF30683F1830683760074628
:101C4000FEF758FC691C00083D68009C019804449C
:101C5000083E356077602746FFF794FF3F1D0098E8
:101C6000001D0090F0D703B080CE00BD2802000810
:101C700000B500BFFFF752FC100000202C1900082F
:101C8000C453454C4620202000B500BFFFF765FC3B
:101C900000000000F0160008C253302000B500BF5D
:101CA000FFF75BFC18000000A80E0008C2523020AD
:101CB00000B500BFFFF751FC1C000000801C0008AD
:101CC000C42354494220202000B500BFFFF745FC43
:101CD000200000004C190008C4275449422020204D
:101CE00000B500BFFFF739FC24000000B013000866
:101CF000C33E494E00B500BFFFF72FFC280000008F
:101D00007C190008C8584F4E2F584F4646202020B7
:101D100000B500BFFFF721FC2C0000007413000881
:101D2000C74543484F494E4700B500BFFFF715FC74
:101D300030000000440F0008C34F555400B500BFE9
:101D4000FFF70BFC34000000301B0008C442415375
:101D50004520202000B500BFFFF7FFFB3800000042
:101D6000D81C0008C3484C4400B500BFFFF7F5FB82
:101D70003C000000EC080008C748414E444C455266
:101D800000B500BFFFF7E9FB40000000C01C0008E1
:101D9000C344504C00B500BFFFF7DFFB4400000018
:101DA000AC1C0008C54F50564543202000B500BF6D
:101DB000FFF7D3FB48000000F8140008C54950564F
:101DC0004543202000B500BFFFF7C7FB4C000000D3
:101DD00000B500BFFFF7C1FB50000000801B0008EA
:101DE000C350414400B500BFFFF7B7FB98000000A7
:101DF000A41D0008C2424C2000B500BFFFF75BFBEA
:101E000020000000641D0008C546454E43452020C3
:101E100000B500BFFFF782FB140000204C1D000836
:101E2000C244502000B500BFFFF778FB1800002027
:101E3000F41D0008C252502000B500BFFFF76EFB32
:101E40001C00002000B500BFFFF768FB2000002049
:101E500000B500BFFFF762FB24000020081E000849
:101E6000C358445000B500BFFFF758FB28000020BE
:101E700000B500BFFFF752FB2C00002000B500BFEB
:101E8000FFF74CFB3000002000B500BFFFF746FB1A
:101E900034000020041D0008C44C4153542020206D
:101EA00000B500BFFFF73AFB3C00002000B500BFC3
:101EB000FFF76EFB4000002000B500BF00F05DFFA3
:101EC000C41E00084C00002000B500BFFFF726FB31
:101ED00090000020BC1D0008C34B45595D46ED6CC9
:101EE0002D6800B501200543A84700BD781D0008F6
:101EF000C44B45593F2020205D46ED6C6D6800B510
:101F000001200543A84700BD70150008C4454D4990
:101F1000542020205D46696B491C69635D46AD6CA9
:101F2000AD6800B501200543A84700BDAC1200080C
:101F3000C4545950452020205D46696BC919696316
:101F40005D46AD6CED6800B501200543A84700BDB6
:101F5000981C0008C24352205D46002068635D461D
:101F6000AD6C2D6900B501200543A84700BD0000F8
:101F7000301F0008C553504143452020361F3760AD
:101F8000202700B5FFF7C6FF00BD00000C1F0008AA
:101F9000C653504143455320002F00DC0027361F15
:101FA0003760002700B500BFFEF7A4FABF1F000886
:101FB000FFF7E4FF0098401C0090F9D703B000BD84
:101FC000201D0008C44845524520202003480568CC
:101FD0002D68361F37602F4670470000280000200C
:101FE000381D0008C34F5247024805682F6080CE55
:101FF0007047000028000020201E0008C5414C4CFE
:102000004F542020034805682968C919296080CEEB
:102010007047000028000020901D0008C552484568
:102020005245202002480568361F37602F4670470A
:102030001C000020741F0008C652414C4C4F542015
:1020400002490868C019086080CE70471C00002053
:10205000541F0008C3524F4D0148024908607047A1
:10206000180000202800002054200008C352414DD1
:1020700001480249086070471C0000202800002029
:1020800004480568361F37602F4600B5FFF7E4FFA8
:1020900000BD00002800002001490F6080CE70477D
:1020A00028000020064805680648854201D0002522
:1020B00001E001256D42361F37602F467047000052
:1020C0002800002018000020FC1F0008C5414C49D2
:1020D000474E202000B5FFF779FFFF1C03218F43F7
:1020E000FFF782FF00BD0000A81B0008C12C2020C4
:1020F00000B5FFF76BFFFFF745FD361F376004277C
:10210000FFF780FF00BD0000901F0008C2572C2081
:1021100000B5FFF75BFFFFF721FD361F3760022791
:10212000FFF770FF00BD00006C200008C2432C20A8
:1021300000B5FFF74BFFFFF7FDFC361F37600127A7
:10214000FFF760FF00BD202002480568361F37609A
:102150002F4670473C0000200448056804490D6084
:102160002D1F2D6801490D60704700003C000020C4
:10217000900000200248056802490D607047000089
:10218000900000203C000020581B0008C446494E27
:10219000442020207D1C3C78083E3560776027462F
:1021A00000B5FEF731FE3D78002D26D0154D2C46AA
:1021B0000834083E346077602F4600BFFEF78EF982
:1021C000FB2100087D1C3C78009B019803441B68A0
:1021D0000C3E34607560B7601F46FEF74FFF002F5E
:1021E00000D180CE04D003B031687160361D00BDCF
:1021F0000098001D0090E5D703B0361F3760002718
:1022000000BD000034000020E01D0008C52E4E4136
:102210004D4520207D1C3F781F200740361F35602C
:1022200000B5FFF789FEFFF7A9FE00BD361F376036
:10223000202700B500F0A0FC7D1C3F780C3E3560E7
:102240007760B560FEF7E0FD3A4805680C3E376000
:10225000F1687160B7602F46FEF710FF002F80CE47
:102260000ED0FEF7CDFEFFF777FEFFF7D3FF00F0AD
:10227000A3F80D6973207265646566696E656420F4
:10228000FFF728FF35682D78ED192A480468236880
:102290005B1E1D40AD00241D64192568083E346096
:1022A00077602F46FFF724FFFFF790FE31680F603D
:1022B00077680836FFF78AFE1F490F607068471E6F
:1022C00035686D1C1D480468002CEFF3008001B4D4
:1022D00077602F46361D01BC80F3008803D0361F7F
:1022E0003760802702E0361F3760C02771680878A2
:1022F0003843087011490020086070683168471839
:10230000706877600746361DFEF7F4F82D23000845
:10231000009D019805442D88361F37602F46FFF732
:10232000F7FE0098801C0090F2D703B0FFF7D2FEB2
:1023300000BD0000300000203C0000200000002014
:10234000002F80CE00B506D0074805682D1D361F2A
:1023500037602F4604E005480568361F37602F4672
:10236000FFF7C6FE00BD0000180000201C00002082
:1023700000B5FEF78DFF00BD00B5FEF789FF7D1C9F
:102380003F78361F356000BD00B5FEF781FF30682D
:102390000028EFF3008001B4361D01BC80F30088F3
:1023A00005D05D462F65034F00F038F800E080CE81
:1023B00000BD0000FEFFFFFF00B5FEF769FF7D1CBA
:1023C0003F78361F3560FFF7B7FD00BD38200008A5
:1023D000C543415443482020361F3760374600B577
:1023E00080B44F4680B45F463F6C80B46F465D4614
:1023F0002F6435687768083601200543A84720BC5C
:102400005C46256401B001B0361F3760002700BD6F
:102410000C210008C55448524F572020002F00B50A
:1024200001D180CE00BD5D462D6CAD4620BC5C4622
:10243000256420BCA94620BC80B42F463E1C80CE1B
:1024400080BC00BD2C210008C63F5448524F572085
:1024500030680028EFF3008001B4361D01BC80F322
:10246000008800B502D0FFF7D9FF00E080CE00BDA4
:102470001C2000088641424F5254222000B500F033
:10248000B5FC361F3760034FFEF726FF00F01AFF3A
:1024900000BD000088230008601E0008C34845589E
:1024A0005D461020A86370479C240008C74445433C
:1024B000494D414C5D460A20A8637047C41F00087F
:1024C000C4484F4C442020205D460448E96B09185D
:1024D000E9635D46ED6B2F7080CE7047FFFFFFFF15
:1024E000341E0008C12320205D46AD6B361F3760C7
:1024F0002F4600B5FEF7E6F970680928EFF3008073
:1025000001B43D46776831687160356001BC80F385
:10251000008800DDFF1D3037FFF7D6FF00BD00004B
:1025200048240008C223532000B500BFFFF7DCFF9A
:1025300035683D43002DF9D100BD0000D81E0008CC
:10254000C23C23205D4698355C46E5637047000039
:1025500024250008C2233E205F46FF6B5D46983568
:10256000ED1B37602F46704774240008C3442E5279
:1025700000B580B437687068316871603060FEF70C
:102580006FF8FFF7DFFFFFF7CFFF70680028EFF36A
:10259000008001B431687160361D01BC80F3008891
:1025A00004D5361F37602D27FFF78EFFFFF7D4FFC6
:1025B00020BCED1B361F37602F46FFF7EDFCFFF701
:1025C000BBFC00BDCC200008C2442E20361F376063
:1025D000002700B5FFF7CCFFFFF7D0FC00BD0000DF
:1025E000F01E0008C12E2020FD17361F37602F4631
:1025F00000B5FFF7EBFF00BD6C250008C2552E208B
:10260000361F3760002700B5FFF7E0FF00BD000070
:10261000981E0008C22E522000B580B43168CF1732
:1026200020BC361F37602F46FFF7A2FF00BD000019
:10263000F01C0008C62B4449474954205D46AD6B49
:10264000361F7168316077602F4600B5FEF72EF8AF
:102650005F46BF6B3568B16831607168B1607560A5
:10266000FEF724F8FDF7C2FF5D466D6C6D1C03D0CC
:102670005D46696C491C696400BD00005425000872
:10268000C73E4E554D424552083E376077600027A1
:1026900000B500BFFDF72EFFF926000835682D783C
:1026A000361F37602F46FEF7A1FB5D46AD6B361F28
:1026B00037602F46FEF7F6FC002F01D0002701E01F
:1026C00001277F42002F80CE01D002B000BD3168CB
:1026D000706801B402B40836FFF7B0FF20BC10BC2C
:1026E0000123ED1A1B19083E336077602F460098CE
:1026F000401C0090D2D703B000BD20205D462F487B
:10270000686435682D782D2D01D0002501E0012564
:102710006D4200B520B4002D04D001257F1B306828
:102720002D183560012F03DA01B00027361D00BDDA
:10273000083EB1683160002171600021B16000BFC6
:10274000FFF7A2FF002F22D001257F1B30682D1834
:10275000356000BF3068451E2D783A2DEFF30080BC
:1027600001B4361F37602F4601BC80F3008801D1C9
:1027700080CE0BE02E2F04D15F460020786480CEFF
:1027800004E001B00027103600BD80CED8E780BC41
:10279000002FEFF3008001B47768083601BC80F3A6
:1027A000008801D0FDF73AFF5D466D6C002D01D524
:1027B000012702E0361F3760022700BDFFFFFFFF41
:1027C00000B500BF35682D78242DEFF3008001B4EB
:1027D000361F37602F4601BC80F300880AD10127DD
:1027E0003168CD1B70683F1877602F46361DFFF7A4
:1027F00057FE1BE0232F0AD101273168CD1B7068DB
:102800003F1877602F46361DFFF754FE0EE0252F48
:102810000BD101273168CD1B70683F185C46022040
:10282000A06377602F46361D00E080CE00BD00001B
:1028300034260008C8494E54454745523F202020C1
:102840007D1C3F78002FEFF3008001B4361F356008
:1028500001BC80F3008800B510D0083EB16831603B
:102860007760FEF7D1FA5D46AD6B20B4FFF7A8FFA5
:10287000FFF744FF20BC5C46A56301E00027361D3E
:1028800000BD000080260008C74E554D4245523F0E
:1028900000B500BFFEF77CFE940000205D466D6B26
:1028A000361F37602F46002F00D180CE00B50FD0E5
:1028B000361F37600827FFF72DFBFFF75FFB361F3A
:1028C00037600827FFF726FB7F1E5D466F6380CECB
:1028D00000BD2020002F01D1002501E001256D421F
:1028E0005C46246B002C01D1002401E001246442E9
:1028F0002C4000B506D0FFF7D1FF7F1E361F376092
:10290000024F02E0361F3760002700BDFFFFFFFFC8
:10291000306838705F463F6B002F80CE00B502D024
:10292000FFF7F8FA00E080CE00BD00001426000892
:10293000822E2220361F3760034F00B5FEF7CCFCF5
:1029400000F0C0FC00BD0000B8230008C825000846
:10295000C2242E207D1C3F78361F356000B5FFF75E
:10296000EBFA00BDFC250008C64143434550542006
:10297000002F00B501D1361D00BD5D46ED6A002D6A
:1029800004D0361F37601127FFF7C4FA30683F18AC
:10299000361F376077680021716000BFFDF7AAFD20
:1029A0003F2A0008FFF79AFA082F03D180CEFFF7DD
:1029B00091FF3EE0092F0CD1009F01980744361F7C
:1029C00020213160FFF7A4FF7F1C361F37600127ED
:1029D0002FE00A2F01D100272BE00D2F0AD1009FF5
:1029E00001980744361F20213160FFF791FF02B0A4
:1029F00000BD1EE00C2F0AD1009F01980744361F2E
:102A000020213160FFF784FF02B000BD11E07F2F6D
:102A100003D180CEFFF75EFF0BE0009D01980544D7
:102A2000361F37602F46FFF773FF7F1C361F376056
:102A300001270098C019009080CEB3D703B05D463F
:102A4000ED6A002D04D0361F37601327FFF762FAB6
:102A500000BD000000B500BFFEF760FD980000203B
:102A600002480568361F37602F46704798000020DF
:102A70005D466D6A5C46246A083E3560776027468D
:102A80007047000050290008C55155455259202073
:102A90000020094908605D466D6A083E3560776030
:102AA000FF2700B5FFF764FF5D462F625F460020F9
:102AB000B86280CE00BD0000980000208828000881
:102AC000C55041525345202000B580B480CEFFF759
:102AD000CFFF5D46AD6A7F1B30682D1810BC083EE5
:102AE00037607560B5602746FEF74CF880B43168F2
:102AF00070680F1A20BC002D01D1002501E00125CE
:102B00006D427D1B5C46A16A4919A162361D00BD5C
:102B100000B580B480CEFFF7ABFF5D46AD6A7C1B8D
:102B200030682D18009B083E34607560B7601F4602
:102B3000FEF714F820BC083E3760B16871602F467C
:102B4000FEF720F880B4316870680F1A20BC002DA1
:102B500001D1002401E0012464426419B1680C1B16
:102B60005D46AC627168B160083600BDAC240008F7
:102B7000C4574F524420202000B5FFF7C9FF064834
:102B80000568361F37602F46FEF762F90248056870
:102B9000361F37602F4600BD1C00002000B5FFF730
:102BA000ABF9002F00D100BDFFF798F9202F80CEA0
:102BB00008D180CEFFF792F9202F01D1002701E044
:102BC00001277F4200BD2020002F00B501D0014821
:102BD0003F1A00BD000000085D46983504480468AF
:102BE0002468A4006419083E346077602F4670475B
:102BF00034000020083E002131607760002700B5D6
:102C0000FFF7EAFFFDF76AFC352C0008009D0198EC
:102C100005442D68AF4208D2009F01980744009DEB
:102C2000019805442D6837602F460098001D0090DC
:102C3000ECD703B0002F01D001483F1800BD80F34E
:102C400000000008104805682D1D361F37602F460C
:102C500000B5FFF7C1FF00BFFDF740FC852C000861
:102C60003D68361F37602F46FFF7AEFF009D019885
:102C700005442F6037683F1D361D0098001D0090E9
:102C8000EED703B080CE00BD34000020C024000881
:102C9000C5574F524453202000B5FFF75DF9FFF7A9
:102CA0008BFB06574F52445320000000FFF754F9A6
:102CB000FFF7C8FFFFF79EFF361F3760FFF76EFF75
:102CC000002F01D0002701E001277F4231680F402B
:102CD000EFF3008001B47768083601BC80F3008808
:102CE00012D05D466D6B402D01DDFFF735F9361FC3
:102CF0003760FFF78FFA3F1F3F68FFF765FF3168C6
:102D00000F6077680836D5E77768083600BD0000A1
:102D100034280008C44D4F564520202000B580B40B
:102D2000316870680F1A009DBD4280CE06D920BC64
:102D3000361F37602F46FEF73BF805E020BC361FF4
:102D400037602F46FEF716F800BD00001424000877
:102D5000C5444550544820205D46AD69361F376054
:102D60002F46361F376037463168CF1B3F1F37600D
:102D7000042700B5FDF774FD00BD7046401E0268D3
:102D80001268014B1A6000BD340000203068874291
:102D900001D1002701E001277F423760024F00B5D3
:102DA000FFF756FB00BD0000EAFFFFFF361F37604C
:102DB000374602490F6080CE704700002400002093
:102DC000361F3760374607480568BD4201D10027E6
:102DD00001E001277F42361F3760034F00B5FFF740
:102DE00037FB00BD24000020EAFFFFFF074805680D
:102DF000002D01D0002501E001256D42083E35601F
:102E00007760034F00B5FFF723FB00BD2C000020C7
:102E1000F2FFFFFF04480568083E35607760034F06
:102E200000B5FFF715FB00BD2C0000206DFEFFFF75
:102E3000882A000882444F2000B5FFF7D7FFFEF72D
:102E4000D1FC361F3760032700BD0000E41F0008D7
:102E5000833F444F00B5FFF7C9FFFEF7D1FC361F93
:102E60003760032700BD000030290008844C4F4F15
:102E70005020202000B5FFF7B9FF361F3760032729
:102E8000FFF784FFFEF7CAFC00BD00006C2E0008AF
:102E9000852B4C4F4F50202000B5FFF7A7FF361F62
:102EA00037600327FFF772FFFEF7C6FC00BD000086
:102EB0006829000885424547494E202000B5FFF7A4
:102EC00095FFFEF735FC00BD342E000885414741D3
:102ED000494E202000B5FFF789FFFEF733FC00BD07
:102EE0008C21000885554E54494C202000B5FFF731
:102EF0007DFFFEF733FC00BD902C00088557484944
:102F00004C45202000B5FFF771FFFEF73FFC30680D
:102F10003760074600BD0000D023000886524550A8
:102F20004541542000B5FFF761FFFEF70BFCFEF7AB
:102F3000F3FB00BD702B00088249462000B5FFF767
:102F400055FFFEF723FC00BD1C2F000884544845A4
:102F50004E20202000B5FFF749FFFEF7DDFB00BD46
:102F6000502D000884454C534520202000B5FFF724
:102F70003DFFFEF7FFFB306837600746FEF7CCFBEE
:102F800000BD0000B42E000884434153452020209A
:102F900000B5FFF72BFF06480568361F37602F4640
:102FA000FEF75EFCFFF702FF361F3760042700BD07
:102FB00024000020142D0008824F4620361F376061
:102FC000042700B5FFF7E2FEFEF758FC361F376016
:102FD000052700BD502E0008833F4F46361F37603F
:102FE000042700B5FFF7D2FEFEF794FC361F3760CA
:102FF000052700BDE42E000885454E444F4620209D
:10300000361F3760052700B5FFF7C0FEFEF742FC0C
:10301000361F3760042700BDFC2E000887454E444C
:1030200043415345361F3760042700B5FFF7AEFE16
:10303000FEF752FC01490F6080CE00BD2400002045
:10304000CC2E0008884E455854434153452020203B
:10305000361F3760042700B5FFF798FEFEF748FCDF
:1030600001490F6080CE00BD24000020642F0008BD
:10307000875245435552534505480568361F37600A
:103080002F4600B5FDF7ACFFFEF726F900BD0000A6
:103090003C000020361F376037465D46AD69BD42B3
:1030A00001D3002701E001277F42361F3760024F1E
:1030B00000B5FFF7CDF900BDFCFFFFFF002F01D0E9
:1030C000002701E001277F42361F3760024F00B51D
:1030D000FFF7BEF900BD0000F3FFFFFF4C2F000813
:1030E00088504F5354504F4E45202020361F376094
:1030F000202700B5FFF740FDFFF74CF8361F37607B
:10310000FFF7DCFF0120C74280CE04D100F060F859
:10311000361F3760014FFEF7DFF800BDD8120008F8
:10312000C02A00088253222010480568002D00B5EF
:1031300007D0361F37600E4FFEF7CEF800F0C2F80A
:1031400013E0361F37602227FFF7BEFC5D46983537
:10315000361F37602F46FDF77BFE5D4698356C1CA9
:103160002D78083E346077602F4600BD2C0000208B
:103170007823000824310008824322200F48056884
:10318000002D00B507D0361F37600D4FFEF7A4F8AD
:1031900000F098F810E0361F37602227FFF794FC04
:1031A0005D469835361F37602F46FDF751FE5D4668
:1031B0009835361F37602F4600BD00002C000020D8
:1031C000702300080C220008874C49544552414C9A
:1031D00000B5FEF7E7FA00BD882F0008C443484158
:1031E00052202020361F3760202700B5FFF7C4FC8F
:1031F0007F7800BDB82F0008865B434841525D20B0
:1032000000B5FFF7F3FDFFF7EDFFFFF7E1FF00BDAE
:103210001C300008815B20200149002008607047B5
:103220002C00002040250008C15D2020024901201B
:1032300040420860704700002C000020E030000889
:10324000C1272020361F3760202700B5FFF794FCE8
:10325000FEF7A0FFFFF732FF00BD00002832000894
:10326000835B275D00B5FFF7EDFFFFF7B1FF00BD02
:10327000E4240008895B434F4D50494C455D2020B4
:1032800000B5FFF7DFFFFEF727F800BD703000083C
:1032900081282020361F3760292700B5FFF76CFCF6
:1032A00080CE00BDEC200008815C2020361F3760F6
:1032B000002700B5FFF760FC80CE00BD7432000827
:1032C000C2222C20361F3760222700B5FFF754FC9E
:1032D0003D786D1CED19361F356000BFFDF70AF90A
:1032E00001330008009D019805442D88361F376082
:1032F0002F46FEF70DFF0098801C0090F2D703B018
:10330000FEF7E8FE00BD202000B520BCE41D03212F
:103310008C4310B42D682F6080CE00BD382F00087C
:103320008249532000B5FFF78DFFBF680848056844
:10333000002D07D0361F3760064FFDF7CDFFFEF793
:10334000D7FE03E0306838607768083600BD0000BB
:103350002C000020083300089032000884455849AA
:103360005420202000B5FFF741FDFEF731FA00BDE3
:1033700014320008813B202000B5FFF737FDFFF72E
:103380001FFDFEF725FAFEF7F5FEFFF745FF00BD2E
:10339000D82F0008C9494E54455250524554202058
:1033A00000B500BFFFF776FE361F37602027FFF716
:1033B000E3FB3D78002D3FD0FEF7ECFE002F00D15F
:1033C00080CE13D0002F01D4002701E001277F42D7
:1033D0001A4805683D4080CE02D0FDF77DFF04E02D
:1033E0003D4680CE01200543A84724E0FFF750FA70
:1033F000002F01D0361F3760FFF760FE0F480568C9
:10340000002D17D0012F03D180CEFEF7CBF910E0AD
:10341000022F08D1776831687160361DFEF7C2F956
:10342000FEF7C0F905E0361F3760054FFEF7F6FFDF
:1034300080CE00E080CEB5E780CE00BD2C0000201D
:10344000F3FFFFFFA8320008C84556414C554154D0
:10345000452020205D466D6A00B520B45D462D6A8A
:1034600020B45D46AD6ABD4201DB002701E00127C3
:103470007F421048056820B45D462F625F46306881
:1034800078620D480B4908605F460020B8620B4F18
:10349000361DFEF7A1FF20BC06490D6020BC5C462E
:1034A000A56220BC5C46256220BC5C466562FEF7D6
:1034B000B5FF00BD98000020FFFFFFFFA03300080C
:1034C00000B500BF002F01D180CE29E00120C74206
:1034D00001D180CE24E00220C74208D15F463F6D73
:1034E0007D1C3F78361F3560FEF726FD18E00D2065
:1034F000C7420AD180CEFEF75FFF0C697320756E5C
:10350000646566696E6564000AE0FEF755FF0B545A
:1035100068726F7720636F6465200000FFF764F8BE
:1035200000BD000078310008C451554954202020C6
:103530005D460020E8625D4601204042286300208D
:103540002E49086000B5FFF767FE00BF5D46ED69D4
:10355000AD465D462D6B002D01D0FEF7FDFCFFF75B
:1035600097FA361F3760264FFEF736FF002F24D11B
:1035700024480768002F01D0002701E001277F427F
:103580005D462D6B002D01D1002501E001256D4226
:103590003D4080CE10D0FEF70FFF03206F6B000080
:1035A000FFF7DAFB002F00D180CE05D0FEF704FF35
:1035B000012D0000FFF718F81EE0FFF781FF5D46C0
:1035C000AD69361F37602F463E1C80CEFFF724FEC4
:1035D000FEF7C2FCFFF74CFAFEF7AEFCFEF7BCFCB0
:1035E0005D46AD6A6D1E361F37602F46FEF7D4FC70
:1035F000FEF7E2FE015E0000A8E700BD9800002093
:10360000A03300082C000020A44900088005000811
:1036100074330008C9434F4C44434841494E20206D
:1036200000B500BFFDF77AFF9C000020DC310008E8
:10363000C64154434F4C442000B5FEF74BFDFEF706
:10364000C5FC054805682F6003490F600027FEF799
:103650004FFDFEF74DFD00BD9C000020C03200086C
:10366000CD57414C4B434F4C44434841494E202099
:10367000361F3760054F00B5002F05D07D6801204B
:103680000543A8473F68F7E780CE00BD083600082D
:10369000361F3760004F01E0807D000800B500BF95
:1036A0003D68002D0FD03D460C353C687B680C3ED4
:1036B00033607560B7602746FDF75CFB3D68ED1928
:1036C0000C352F46ECE75F461837083E3760144943
:1036D00071601027FDF74EFB5D46AD69361F376000
:1036E0002F463E1C80CE5D460E4868625D46002037
:1036F00028640C3E0C4931600C497160B76010279A
:10370000FDF738FB00200A490860FEF7D3FE094D9B
:1037100009490D6009490D6000200949086000BD94
:10372000F8010008203C00201400002018020008C6
:10373000980000204C0000203400002030000020C1
:1037400038000020C8310008C52E465245452020CB
:1037500000B5FEF701FC1548056815494D1B361FDD
:1037600037602F46FEF74CFFFEF726FE1062797495
:103770006573206672656520466C617368000000A1
:10378000FEF7EAFB04F0DAFA0A4805687F1BFEF749
:1037900037FFFEF711FE0E6279746573206672655D
:1037A000652052414D00000000BD000018000020BF
:1037B00000F001081C0000205C330008C6434F4D98
:1037C0004D495420002F00B500D1074F0120074379
:1037D00006490F60083E7C27054931600549716044
:1037E000FEF718FA00BD0000800500084000002028
:1037F00000F8010814000020F82F0008C5454D50BE
:1038000054592020083E0849316077607C2700B574
:10381000FEF7CEF9083E054931607760044FFEF7A8
:10382000C7F900F081F800BD00F8010800C00008E9
:1038300000F0000030360008C4434F4C44202020E4
:1038400000B5FFF725FF01F0D7FC01F0DDF95D467B
:10385000AF6480CE01F0D8F95D46EF6480CE01F010
:103860000FFF0C3E2749316027497160B7607C2704
:10387000FEF7D0F9254805680120C54201D1002492
:1038800001E001246442002D01D1002501E0012561
:103890006D4225400ED01E4805681E480468AC42A3
:1038A00008D10C3E1849316018497160B7607C2717
:1038B000FDF760FAFEF70EFC174805682D68012039
:1038C000C54201D0FFF79EFFFFF7D2FEFEF744FB93
:1038D00002F0E0F9FFF73CFFFEF7E8FAFEF73CFBE9
:1038E000FEF73AFBFEF768FD0420206F6B00000036
:1038F0005D46AD69361F37602F463E1C80CEFFF710
:1039000017FE00BD00F001081400002000F80108B7
:10391000280200087CF80108180000204032000846
:10392000C65245424F4F542072B6054901200D68DA
:1039300005430D6003480449086000B5FEE700BD7B
:1039400024100240CCCC000000300040F0B54046CE
:10395000494652465B460FB46946F0398B460A1C0D
:10396000F03A95460E46083E341F8C616846C861A1
:10397000FCF706FE6946F031F0318D460FBC8046FB
:10398000894692469B46F0BD902E0008C7494E548A
:103990003E4249541F253D400124AC407F09BF00F1
:1039A000361F346070470000FC370008C5454E499B
:1039B0004E5420200F2F00B50BD9103FFFF7EAFF20
:1039C00005483F1805483F18306838607768083662
:1039D00000BD80CE00BD000000E000E0000100005E
:1039E000AC390008C6444953494E54200F2F00B546
:1039F0000BD9103FFFF7CEFF05483F1805483F1889
:103A0000306838607768083600BD80CE00BD0000A1
:103A100000E000E080010000BC370008C6534554B8
:103A2000505249200F2F00B509D9103F05483F18C3
:103A300005483F18306838707768083600BD80CE7A
:103A400000BD000000E000E0000400002039000894
:103A5000C55357494E5420200F2F00B50BD9103FA6
:103A6000FFF798FF05483F1805483F183068386051
:103A70007768083600BD80CE00BD000000E000E0A1
:103A800000020000503A0008C92F415050465241F0
:103A90004D45202000B500BFFDF70DFD20000000C2
:103AA00020330008C64558412E52302000B500BFD3
:103AB000FFF7FFFF00000000A43A0008C645584188
:103AC0002E52312000B500BFFFF7FFFF04000000B9
:103AD000BC3A0008C64558412E52322000B500BFFE
:103AE000FFF7FFFF08000000D43A0008C645584120
:103AF0002E52332000B500BFFFF7FFFF0C0000007F
:103B000014360008C74558412E52313200B500BF67
:103B1000FFF7FFFF10000000043B0008C7455841B5
:103B20002E52313400B500BFFFF7FFFF1400000034
:103B3000EC3A0008C64558412E50432000B500BF5E
:103B4000FFF7FFFF180000001C3B0008C745584165
:103B50002E50535200B500BFFFF7FFFF1C000000BE
:103B60001C3A0008CA2F4D41494E4652414D45204E
:103B700000B500BFFDF79FFC24000000343B0008A7
:103B8000C645584D2E52342000B500BFFFF7FFFF49
:103B900000000000803B0008C645584D2E523520DD
:103BA00000B500BFFFF7FFFF04000000983B0008CE
:103BB000C645584D2E52362000B500BFFFF7FFFF17
:103BC00008000000B03B0008C645584D2E52372073
:103BD00000B500BFFFF7FFFF0C000000C83B000866
:103BE000C645584D2E52382000B500BFFFF7FFFFE5
:103BF00010000000E03B0008C645584D2E52392009
:103C000000B500BFFFF7FFFF140000004C3B0008A9
:103C1000C745584D2E52313000B500BFFFF7FFFFAA
:103C200018000000103C0008C745584D2E52313195
:103C300000B500BFFFF7FFFF1C000000E4250008EF
:103C4000CA45584D2E4558435245542000B500BF33
:103C5000FFF7FFFF2000000044300008C72F455841
:103C60004441544100B500BFFDF725FC140000009D
:103C7000403C0008CA4558442E523133464C54202B
:103C800000B500BFFFF7FFFF000000008C390008FF
:103C9000CB4558442E5231334D41494E00B500BFFB
:103CA000FFF7FFFF0400000048370008CE455844E6
:103CB0002E52313350524F434553532000B500BF6D
:103CC000FFF7FFFF08000000F8310008CC4558441A
:103CD0002E523133535441544520202000B500BFAB
:103CE000FFF7FFFF0C000000743C0008CA45584471
:103CF0002E4C524D41494E2000B500BFFFF7FFFF4B
:103D000010000000F83B0008C645584441544120CB
:103D100000B500BFFDF7CFFB4C360020164BEFF38C
:103D200008805860EFF30981996072461A61042097
:103D3000024201D1586800E0986818604046494640
:103D400052465B460FB5F0B40B4B6846D860F8B0EE
:103D50006846F03083460646083E341F8461694653
:103D6000C161FCF70DFC78B0F0BC0FBC8046894601
:103D700092469B4600BD00004C360020AC3C00083B
:103D8000C52E4954454D20203D68361F37602F46CB
:103D900000B501F0BFFAFEF7F1F83F1D00BD0000CD
:103DA00060360008C62E4954454D5320361F3760F3
:103DB000002700B5FCF79EFBCB3D0008FFF7E4FFB2
:103DC0000098401C0090F9D703B000BD643B000888
:103DD000C84150504954454D5320202002480568A1
:103DE000361F37602F4670474C3600205C3C000879
:103DF000C94D41494E4954454D532020024805685C
:103E0000361F37602F467047583600203838000874
:103E1000C64150505253502000B5FFF7DFFF203706
:103E200000BD0000103E0008C641505050535020C5
:103E300000B5FFF7E3FFBF6800BD0000F03D0008DC
:103E4000C54150505550202000B5FFF7D7FFFF69FE
:103E500000BD0000283E0008C6415050544F53207A
:103E600000B5FFF7CBFFFF6800BD0000403E000833
:103E7000C54150505043202000B5FFF7AFFFBF6948
:103E800000BD0000583E0008C92E464C5446524121
:103E90004D45202000B5FFF7A1FFFEF75DF8FEF7C6
:103EA0008BFA113D3D3D20526567697374657273ED
:103EB000203D3D3DFEF750F8FEF77EFA0650535286
:103EC000203D2000FD69361F37602F4601F022FAA1
:103ED000FEF742F8FEF770FA06523020203D20002F
:103EE000083E376077600427FFF760FF80CEFFF75A
:103EF00085FFFEF731F8FEF75FFA06523420203DC9
:103F000020000000361F37600427FFF74FFFFEF741
:103F100023F8FEF751FA06523820203D2000000019
:103F2000361F37600427FFF741FF80CEFFF756FFAB
:103F3000FEF712F8FEF740FA06523132203D20001B
:103F40003D461035361F37602F46FFF71DFF376897
:103F5000203701F0DFF9FEF711F81437361F37600C
:103F60000227FFF723FF80CE00BD0000803D000840
:103F7000C54E414D453F2020FD1C03218D43AF42DE
:103F800000B501D0002700BD7D1C3F789F243C4038
:103F9000103E812131607460B760F560A027FCF7A6
:103FA00047FA002F80CE02D10027361D00BD1F200A
:103FB000074030683F18306837600746FCF79AFAC8
:103FC000F73F0008009D019805442D780C3E212103
:103FD00031607560B7607F27FCF72AFA002F80CE2A
:103FE00004D103B0361F3760002700BD0098401C85
:103FF0000090E7D703B0361F3760014F00BD0000C7
:10400000FFFFFFFFEC3C0008C649503E4E464120F2
:10401000BF1E00B5361F3760FFF7AEFF002F80CE02
:1040200001D17F1EF6E700BD903C0008CD43484516
:10403000434B2D414C49474E45442020FD1C032154
:104040008D43AF4200B50CD0FEF7B6F90D284D698F
:1040500073616C69676E656429200000FF1C032191
:104060008F4300BD703E0008C73F434C4950333278
:1040700030683D1A802D00B510D937688037FDF7BC
:104080006BFFFEF799F913436C69707065642074D7
:104090006F203332206974656D73000000BD00002D
:1040A00068400008C82E52534641554C54202020E9
:1040B00000B5FDF751FFFFF7AFFEFDF74DFFFEF72F
:1040C0007BF906525350203D20000000361F376018
:1040D00001F020F9FDF752FFFFF7B0FFFFF7B4FE44
:1040E000FF69FEF769F90720205230203D200000CB
:1040F000361F376001F00EF9FDF740FFFFF79EFF16
:104100003F1FFDF729FFFEF757F9192D2D2D2052DE
:10411000657475726E20737461636B20686967687B
:10412000202D2D2DFFF7A4FFFCF7E4F98D410008A9
:10413000FDF712FF009D01980544361F37602F469A
:1041400001F0E8F8FDF71AFF009D019805442D687D
:10415000083E356077602F4601F0DCF8FDF70EFF72
:104160000C3E144931607760B760134FFCF760F97B
:10417000002F80CE04D0FFF74BFFFEF74BF800E096
:1041800080CE0098001F0090D2D703B0FDF7E4FE68
:10419000FEF712F9192D2D2D2052657475726E20BF
:1041A000737461636B206C6F77202D2D2D200000C0
:1041B00000BD00003402000800C00008A440000850
:1041C000C82E50534641554C5420202000B5FDF7D1
:1041D000C3FEFFF72DFEFDF7BFFEFEF7EDF806501C
:1041E0005350203D20000000361F376001F092F848
:1041F000FDF7C4FEFFF722FFFFF726FEBF69FEF7BB
:10420000DBF80720205330203D200000361F3760A8
:1042100001F080F8FDF7B2FEFFF710FF3D1D30689A
:10422000854212D277680836FDF796FEFEF7C4F88D
:10423000164461746120737461636B20756E6465EC
:1042400072666C6F7765640000BD3D1D3068854205
:104250000FD177680836FDF77FFEFEF7ADF8104402
:1042600061746120737461636B20656D7074790093
:1042700000BD30683D1AF02D11D977680836FDF77A
:104280006BFEFEF799F815446174612073746163E5
:104290006B206F766572666C6F77656400BDFDF7A5
:1042A0005BFEFEF789F8172D2D2D204461746120E7
:1042B000737461636B2068696768202D2D2D000081
:1042C0003068874221D03F1FFFF7D2FEFCF706F986
:1042D00009430008FDF740FE009D01980544361F84
:1042E00037602F4601F016F8FDF748FE009D019853
:1042F00005442D68361F37602F4601F00BF80098F3
:10430000001F0090E6D703B001E077680836FDF79C
:1043100023FEFEF751F8172D2D2D204461746120E6
:10432000737461636B206C6F77202D2D2D2000003E
:10433000FDF712FEFEF740F80972544F532F523723
:1043400020200000FFF78CFD00F0E4FF00BD00001E
:10435000283C0008C953484F574641554C5420202B
:1043600000B500F051FC03F0F7FC00F09BFBFEF7FA
:10437000A1F8FDF7F1FDFDF7EFFDFEF71DF80A4589
:104380007863657074696F6E20000000EFF3058537
:10439000361F37602F46FEF727F9FEF70DF8036149
:1043A00074200000FFF768FD00F0B4FFFFF772FD16
:1043B000FFF77EFEFFF70AFFFDF7CEFDFDF7FCFFDE
:1043C0001552657374617274696E672073797374C2
:1043D000656D202E2E2E0000FFF7A6FA361F3760DF
:1043E000002700BD164BEFF308805860EFF30981FA
:1043F000996072461A610420024201D1586800E0B7
:10440000986818604046494652465B460FB5F0B47E
:104410000B4B6846D860F8B06846F03083460646D5
:10442000083E341F84616946C161FFF799FF78B087
:10443000F0BC0FBC8046894692469B4600BD0000FA
:104440004C360020164BEFF308805860EFF30981DB
:10445000996072461A610420024201D1586800E056
:10446000986818604046494652465B460FB5F0B41E
:104470000B4B6846D860F8B06846F0308346064675
:10448000083E341F84616946C161FFF769FF78B057
:10449000F0BC0FBC8046894692469B4600BD00009A
:1044A0004C36002048340008CA53454C494F2D5320
:1044B000455231201A4D2C463034103E03213160D4
:1044C00000217160B560F760274600B5FDF74AFA34
:1044D00014487969014379611248B96A8143B96224
:1044E0001148B9690143B9610F48F9688143F9601E
:1044F0000E4801B4009F3F1C083E0D4931600D4934
:104500007160FDF72FFA20BC24350C3E0A4931605A
:104510000A497160B7602F46FDF724FA00BD00001C
:1045200000100240000002000040000000000048AF
:1045300000003C0000002800F00F00001001000007
:10454000A43D0008C450494F3A20202000B5FCF794
:104550007BFF31688D020B482D18361F37602F46C0
:10456000FDF7C6FD0125BD40361F37602F46FDF71C
:10457000BFFD31684D013D432F46361DFDF7B8FDA7
:1045800000BD00000000004894330008C2504120E4
:1045900000B500BFFCF78FFF000000008C4500084D
:1045A000C250422000B500BFFCF785FF01000000AB
:1045B000A0450008C250432000B500BFFCF77BFFB8
:1045C00002000000B4450008C250442000B500BFFE
:1045D000FCF771FF03000000C8450008C2504520E9
:1045E00000B500BFFCF767FF04000000DC450008D1
:1045F000C250462000B500BFFCF75DFF050000007B
:10460000D03D0008C653455450494E203D687F6850
:104610002F8380CE7047000004460008C6434C52EA
:1046200050494E203D687F686F8380CE7047000000
:10463000A8440008C647455450494E203D687F684D
:104640002D693D40002D01D1002701E001277F4267
:10465000012007407047202003200740BD003D4354
:104660002F012F433D023D432F042F43704720204D
:104670000F2007407F000325BD402F4670472020B4
:1046800030683760074600B5FFF7E6FF30683760EF
:104690000746FFF7EDFF35683D40356000BD20203F
:1046A000BD680F200540361F7168316077602F4666
:1046B00000B5FFF7E5FF75682D68316871603760F8
:1046C0002F4600BDF0450008C9495350494E4D4F93
:1046D0004445202000B5FFF7E3FF3F1CFDF742F9FA
:1046E00000BD20200F2007403D013D432F022F43F6
:1046F0003D043D432F46704707253D40AD000F2444
:10470000AC40082007407F08361F346070472020E7
:1047100030683760074600B5FFF7E4FF3068376060
:104720000746FFF7E9FF80B4376871680F4020BC87
:1047300077602F4600BD0000C8460008C9494E50AA
:1047400055544D4F4445202000B500BFFCF7B3FE43
:10475000000000001C460008CA4F55545055544DE7
:104760004F44452000B500BFFCF7A5FE0100000046
:10477000883E0008C641464D4F44452000B500BF65
:10478000FCF799FE02000000083D0008CA414E41B6
:104790004C4F474D4F44452000B500BFFCF78BFE02
:1047A000030000002C400008C74953494E5055549F
:1047B000361F0021316000B5FFF78CFF00BD0000FF
:1047C000CC3C0008C849534F555450555420202024
:1047D000361F0121316000B5FFF77CFF00BD0000EE
:1047E000703F0008CA495346554E4354494F4E2026
:1047F00000B580B4009F361F02213160FFF76AFFC9
:10480000009DAD680F200540361F37602F46FFF72B
:104810007FFF20BC2D682035ED192F46FDF7A2F84B
:1048200000BD0000C4470008C84953414E414C4FE9
:1048300047202020361F0321316000B5FFF74AFFD3
:1048400000BD0000A8470008C7495350494E4F44D7
:1048500030680028EFF3008001B4361D01BC80F3FE
:10486000008800B506D03D687F6869683943696093
:1048700080CE05E03D687F686968B943696080CE95
:1048800000BD00003C470008C9495350494E5055EF
:104890005044202000B5FFF703FF0C37FDF762F806
:1048A00000BD000074470008C94E4F5450554C4C91
:1048B00045442020361F0021316000B5FFF7EAFF94
:1048C00000BD0000883A0008C850554C4C4544557E
:1048D00050202020361F0121316000B5FFF7DAFF9C
:1048E00000BD0000E4390008CA50554C4C45444412
:1048F0004F574E20361F0221316000B5FFF7CAFF27
:1049000000BD0000E4470008CA495350494E5350C7
:104910004545442000B5FFF7C3FE0837FDF722F8F0
:1049200000BD000044450008C84C4F575350454552
:104930004420202000B500BFFCF7BDFD00000000B2
:10494000C8480008CB4D454449554D535045454452
:1049500000B500BFFCF7AFFD0100000028480008CB
:10496000C9484947485350454544202000B500BF39
:10497000FCF7A1FD0300000060490008C8494E494A
:10498000544750494F202020044D054C696921436C
:104990006961A96AA143A962704700000010024042
:1049A00000007E0034570008884900087C49000850
:1049B000C9285345524B45593F292020FF692020E3
:1049C0000740704748480008C8285345524B45598E
:1049D0002920202000B500BFFD6920200540002DC2
:1049E00002D1FCF789FEF7E77F6AFF20074000BD90
:1049F000B0490008C928534552454D495429202043
:104A000000B500BFFD6980200540002D02D1FCF7F4
:104A100073FEF7E73068B8627768083600BD0000BB
:104A2000F4490008C92853455254595045292020BB
:104A3000706831684518706877600746356000B562
:104A4000FBF758FD654A0008009D019805442D7844
:104A5000083E35607760FFF7D3FF0098401C009058
:104A6000F2D703B080CE00BD08400008C7285345E8
:104A700052435229083E0D213160776000B5FFF79F
:104A8000BFFF361F0A213160FFF7BAFF00BD0000EB
:104A900044490008CD2B4641554C54434F4E534F8B
:104AA0004C4520207047000088480008CA28494E1D
:104AB00049542D5345522920002038600020786049
:104AC0000020B8603068F8600C2038600D20386035
:104AD0007768083670470000E8480008C55541521D
:104AE0005431202000B500BFFCF7E5FC0038014040
:104AF000AC4A0008C9494E49542D53455231202033
:104B000000B5FFF7D7FC083E034931607760034FDB
:104B1000FFF7D2FF00BD0000E204000000380140B2
:104B20008C470008C85345524B45593F312020203F
:104B3000361F3760024F00B5FFF740FF00BD000091
:104B400000380140DC4A0008C75345524B455931F3
:104B5000361F3760024F00B5FFF73CFF00BD000075
:104B600000380140244B0008C8534552454D495474
:104B700031202020361F3760024F00B5FFF740FF7D
:104B800000BD000000380140684B0008C853455282
:104B90005459504531202020361F3760024F00B550
:104BA000FFF746FF00BD00000038014058470008ED
:104BB000C653455243523120361F3760024F00B56D
:104BC000FFF758FF00BD0000003801408C4B000883
:104BD000C8434F4E534F4C453120202000B500BFF5
:104BE000FCF769FCE84B0008504B0008304B00080C
:104BF000744B0008984B0008B84B0008484B00085D
:104C0000C7434F4E534F4C4500B500BFFCF753FC14
:104C1000E84B0008004C0008C55541525432202092
:104C200000B500BFFCF747FC0044004034460008D4
:104C3000CA53455232434C4F434B53200F4D2C46E1
:104C40003034103E0E49316000217160B560F7606C
:104C5000274600B5FCF786FE0A4879690143796169
:104C60000848B96A8143B9620648F9690143F961A4
:104C7000044839698143396180CE00BD001002408B
:104C80000000030000000200A8480008C354583286
:104C900000B500BFFCF70FFC9C4C0008000000486A
:104CA000040000000200000028350008C3525832FA
:104CB00000B500BFFCF7FFFBBC4C0008000000483B
:104CC0000800000003000000C8490008CD53455209
:104CD0003246554E4354494F4E532020083E012141
:104CE00031607760054F00B5FFF782FD083E012176
:104CF00031607760024FFFF77BFD00BD9C4C0008E0
:104D0000BC4C0008304C0008CA53454C494F2D5349
:104D10004552322000B5FFF791FFFFF7DFFF00BDDE
:104D2000F44A0008C9494E49542D534552322020B7
:104D300000B5FFF7EFFF083E342131607760024F86
:104D4000FFF7BAFE00BD000000440040D04B000851
:104D5000C85345524B45593F32202020361F3760FB
:104D6000024F00B5FFF72AFE00BD000000440040DE
:104D7000184C0008C75345524B455932361F37600F
:104D8000024F00B5FFF726FE00BD000000440040C2
:104D9000504D0008C8534552454D495432202020FB
:104DA000361F3760024F00B5FFF72AFE00BD000036
:104DB00000440040944D0008C85345525459504592
:104DC00032202020361F3760024F00B5FFF730FE3B
:104DD00000BD000000440040B04B0008C6534552DF
:104DE00043523220361F3760024F00B5FFF742FEB4
:104DF00000BD000000440040B84D0008C8434F4EBD
:104E0000534F4C453220202000B500BFFCF753FB28
:104E1000144E00087C4D00085C4D0008A04D0008B1
:104E2000C44D0008E44D0008744D0008C5554152BA
:104E30005433202000B500BFFCF73DFB0048004084
:104E40008C4C0008C354583300B500BFFCF733FB4B
:104E5000544E000800080048100000004400000004
:104E6000AC4C0008C352583300B500BFFCF723FB1D
:104E7000744E000800080048000800004B000000C5
:104E8000084D0008CA53454C494F2D534552332015
:104E9000154D2C463034103E1449316000217160AC
:104EA000B560F760274600B5FCF75CFD10487969EE
:104EB000014379610E48B96A8143B9620D48F969C5
:104EC0000143F9610B48396981433961361F0A4F43
:104ED00001213160FFF78CFC083E012131607760D1
:104EE000064FFFF785FC00BD0010024000000C00DB
:104EF0000000080000000400544E0008744E000832
:104F0000244D0008C9494E49542D534552332020A1
:104F100000B5FFF7BDFF083E034931607760034FDE
:104F2000FFF7CAFD00BD0000A101000000480040DD
:104F3000FC4D0008C85345524B45593F33202020B3
:104F4000361F3760024F00B5FFF738FD00BD000087
:104F5000004800402C4E0008C75345524B4559337A
:104F6000361F3760024F00B5FFF734FD00BD00006B
:104F700000480040344F0008C8534552454D49543D
:104F800033202020361F3760024F00B5FFF738FD71
:104F900000BD000000480040784F0008C85345524B
:104FA0005459504533202020361F3760024F00B53A
:104FB000FFF73EFD00BD000000480040DC4D00084A
:104FC000C653455243523320361F3760024F00B557
:104FD000FFF750FD00BD0000004800409C4F000856
:104FE000C8434F4E534F4C453320202000B500BFDF
:104FF000FCF761FAF84F0008604F0008404F0008C6
:10500000844F0008A84F0008C84F0008584F0008F8
:10501000C55541525434202000B500BFFCF74BFA6F
:10502000004C0040644E0008C352583400B500BF25
:10503000FCF741FA38500008000000480200000068
:1050400001000000444E0008C354583400B500BFAE
:10505000FCF731FA5850000800080048000400002E
:105060004A000000844E0008CA53454C494F2D5356
:1050700045523420144D154869690143696113484C
:10508000A96A8143A96212486969014369611048AC
:10509000A96A8143A9620D48E9690143E9610B48A6
:1050A000296981432961083E042131607760094FF5
:1050B00000B5FFF79DFB083E002131607760064F89
:1050C000FFF796FB00BD0000001002400000080042
:1050D000000002003850000858500008044F000833
:1050E000C9494E49542D53455234202000B5FFF78D
:1050F000C1FF083E034931607760034FFFF7DCFCD6
:1051000000BD0000A1010000004C0040E04F00087D
:10511000C85345524B45593F34202020361F376035
:10512000024F00B5FFF74AFC00BD0000004C0040F4
:1051300010500008C75345524B455934361F37604D
:10514000024F00B5FFF746FC00BD0000004C0040D8
:1051500010510008C8534552454D49543420202071
:10516000361F3760024F00B5FFF74AFC00BD000054
:10517000004C004054510008C85345525459504502
:1051800034202020361F3760024F00B5FFF750FC57
:1051900000BD0000004C0040C04F0008C6534552FF
:1051A00043523420361F3760024F00B5FFF762FCD0
:1051B00000BD0000004C004078510008C8434F4E2D
:1051C000534F4C453420202000B500BFFCF773F945
:1051D000D45100083C5100081C51000860510008DF
:1051E00084510008A4510008244A0008C8494E49C7
:1051F000542D53455220202000B5FFF781FCFFF7C6
:1052000097FDFFF785FEFFF771FF00BD34510008E1
:10521000C753455442415544361F7068776007466E
:105220000549316000B5FBF71BFB7F1C7F08356823
:10523000EF607768083600BD00D8B8050849000857
:10524000CA49532D434F4E534F4C45205D46AF64E2
:105250005D46EF6480CE704728490008C62E415352
:10526000434949207F2007400C3E20213160776070
:10527000B7607F2700B5FBF7DBF8002F80CE00D1A9
:105280002E27FCF747FE00BD40520008C52E4259AC
:10529000544520205D46AD6B00B520B4FDF700F904
:1052A000361F37600027FDF74DF9FDF71DF9FDF7B3
:1052B0001BF9FDF751F9FCF73FFE20BC5C46A563E6
:1052C00000BD00008C520008C52E574F52442020CC
:1052D0005D46AD6B00B520B4FDF7E2F8361F3760D0
:1052E0000027FDF72FF9FDF7FFF8FDF7FDF8FDF7B3
:1052F000FBF8FDF7F9F8FDF72FF9FCF71DFE20BCD0
:105300005C46A56300BD00005C520008C62E4457F1
:105310004F5244205D46AD6B00B520B4FDF7C0F898
:10532000361F37600027FDF70DF9FDF7DDF8FDF7B3
:10533000DBF8FDF7D9F8FDF7D7F8361F37603A27C5
:10534000FDF7C2F8FDF7D0F8FDF7CEF8FDF7CCF881
:10535000FDF7CAF8FDF700F9FCF7EEFD20BC5C464E
:10536000A56300BD944A0008C444554D5020202038
:105370005D46AD6B361F71683160756000B5FDF735
:105380008FF830683F18306837600746FBF7B2F88F
:105390003D540008FCF7E0FD009D01980544361FD0
:1053A00037602F46FFF7B6FF009D019805442C4655
:1053B0001034083E346077602F4600BFFBF78EF84C
:1053C000E5530008FCF7DAFD009D019805442D78AF
:1053D000361F37602F46FFF75DFF0098401C009096
:1053E000F0D703B0361F37600227FCF7D5FD009DCC
:1053F000019805442C461034083E346077602F46EF
:10540000FBF76CF825540008009D019805442D78A1
:10541000361F37602F46FFF725FF0098401C00908D
:10542000F2D703B0FCF768FD002F80CE01D002B0A8
:1054300000BD009810300090ACD703B05D46AF635C
:1054400080CEFCF789FD00BD28500008C5504455AA
:105450004D5020205D46AD6B361F71683160756020
:1054600000B5FDF71DF83068054603218D437F190F
:1054700037602F46FBF73EF8E5540008FCF76CFD5B
:10548000009D01980544361F37602F46FFF742FF05
:10549000009D019805442C461034083E3460776026
:1054A0002F4600BFFBF71AF8CD540008FCF766FD45
:1054B000009D019805442D68361F37602F46FFF781
:1054C00029FF0098001D0090F0D703B0FCF714FDF1
:1054D000002F80CE01D002B000BD009810300090A7
:1054E000CCD703B05D46AF6380CEFCF735FD00BD81
:1054F000CC4C0008C22E532000B5FCF72DFDFCF764
:105500005BFF032D2D200000FDF726FC002F00D1AE
:1055100080CE16D07F1E361F00213160FAF7DEFFE5
:1055200043550008009D01980544361F37602F46FB
:10553000BF00F759FDF764F80098401E0090F1D7BE
:1055400003B000BD4C540008C94C45444143544984
:105550005645202000B500BFFBF7E0FFA00000206B
:10556000C8520008C73C5449434B533E00B500BFE6
:10557000FBF7D4FFA40000209C510008C554494308
:105580004B53202002480568361F37602F4670476E
:10559000A40000206C4A0008C34C445500B500BF6D
:1055A000FBF789FFA85500080008004840000000EC
:1055B0004600000098550008C34C445200B500BF97
:1055C000FBF779FFC85500080008004800020000FA
:1055D00049000000B8550008C34C444400B500BF62
:1055E000FBF769FFE855000800080048800000004C
:1055F00047000000D8550008C34C444C00B500BF1C
:10560000FBF759FF08560008000800480001000099
:105610004800000054430008C95359535449434BB0
:105620004552202002490868401C0860704700006D
:10563000A4000020F0B54046494652465B460FB4F0
:105640006946F0398B460A1CF03A95460E46083EEC
:10565000341F8C616846C861FFF7E4FF6946F0318A
:10566000F0318D460FBC8046894692469B46F0BD80
:1056700060320008CB53544152542D434C4F434B9E
:10568000054D064868610320286105496C18FF2014
:10569000207062B67047000000E000E06F17000065
:1056A000230D000068500008CA53544F502D434C3E
:1056B0004F434B20024901200D6885430D60704720
:1056C00010E000E0EC510008C54C41544552202048
:1056D00002480568ED192F4670470000A40000201D
:1056E000A8560008C954494D45444F55543F202001
:1056F000044805687F1B002F01D4002701E0012723
:105700007F427047A4000020F8550008C24D532086
:1057100007480568ED192F4600B500BFFBF7ECFF01
:10572000034805687D1B002DF8D580CE00BD01BC67
:10573000A40000201C5A0008805600086455000888
:10574000C42F54434220202000B500BFFBF7B3FE16
:105750001800000018560008C85443422E4C494E09
:105760004B20202000B500BFFFF7FFFF0000000026
:10577000BC510008C75443422E53535000B500BFDC
:10578000FFF7FFFF0400000074560008CA544342AC
:105790002E5354415455532000B500BFFFF7FFFF6F
:1057A0000800000058570008C85443422E4D535279
:1057B0004320202000B500BFFFF7FFFF0C000000D2
:1057C000A8570008C85443422E4D45534720202077
:1057D00000B500BFFFF7FFFF10000000E45600080F
:1057E000C95443422E4556454E54202000B500BFB3
:1057F000FFF7FFFF14000000C8560008C44D4149E0
:105800004E20202000B500BFFBF755FE103F0020C2
:10581000000000000C570008C72850415553452987
:10582000C0B5684659464860096888680028FBD0BA
:105830008B4648688546C0BC01BC86467047000060
:1058400040570008864D554C54493F2000B500BFD5
:10585000FBF70FFFA80000207C550008C653494EF7
:10586000474C45200348044908600020034908606C
:10587000704700008105000808000020A8000020F3
:10588000E0500008C54D554C5449202003480449B8
:105890000860044804490860704700002158000867
:1058A00008000020FFFFFFFFA80000205C58000850
:1058B000C6535441545553205D46AD6801218D4374
:1058C000361F37602F467047B0580008C7524553FF
:1058D000544152540120B9680143B96080CE7047E9
:1058E000C4570008C448414C542020200120B96806
:1058F0008143B96080CE704748500008C453544F6C
:10590000502020205D462D1C361F37602F4600B5E5
:10591000FFF7ECFFFBF7F0FE00BD000002CE012315
:1059200019436A463846F0388546F8610020B86069
:1059300002B401B43946091E083902B4091FB9611D
:1059400068467860954680CE704720205D462D6879
:105950003D605D462F6080CE704720205D462D1C47
:10596000361F37602F4600B53D683068854208D045
:105970003F685D462D1CBD4202D17768083600BDE8
:10598000F2E735682D683D607768083600BD000095
:10599000FC570008C8494E4954494154452020202D
:1059A000361F71683160776000B5FFF7B7FF361FAB
:1059B0003760FFF7CBFF0120B86080CEFBF79CFE7D
:1059C00000BD0000E0570008C95445524D494E4102
:1059D0005445202000B5FFF7C1FFFBF78DFE00BD49
:1059E00044580008CA494E49542D4D554C5449203D
:1059F00000B5FFF737FF083E06493160776018278A
:105A000002F0B6F9034D2D60012003490860FFF74D
:105A10003DFF00BD103F0020183F0020D07C000853
:105A2000F059000874570008C34849535D462D1CBF
:105A30007F1B30683F18361D70470000E45800088F
:105A4000C953454D4150484F52452020361F3760BD
:105A5000082700B5FBF76EFD0B4805680C3E0021DA
:105A6000316000217160B7602F46FBF7B9FA3D46FF
:105A700080CE01200543A8473068386070687860A0
:105A8000B7680C3600BD00003C000020CC58000870
:105A9000C65349474E414C2000B5FBF74FFF3868CD
:105AA000401C38600020786080CEFBF751FF00BDBD
:105AB000905A0008C75245515545535400B500BF90
:105AC000FBF73CFF3D68002D04D1FBF741FFFBF7DE
:105AD00013FEF5E73868401E38605D462D1C7D607A
:105AE00080CEFBF735FF00BD8C570008CA544153E8
:105AF0004B2D434841494E2000B500BFFBF70EFD3A
:105B0000AC00002068530008C45441534B202020AF
:105B10000C4805680C482D18083E356077600B4F1F
:105B200000B5FCF78DFAFBF7C1FCFCF74FFA08480B
:105B30000568361F37602F46FCF7DAFA04490F6014
:105B400080CE00BD1C000020F0010000E00200003B
:105B5000AC000020B45A0008C653544152543A20B5
:105B600000B520BC361F3560FFF71AFF00BD0000EE
:105B7000E4590008C52E5441534B2020361F37608E
:105B8000124F00B53F68002F0ED03D1F2D683068C2
:105B9000854208D10C3F361DFBF732FAFCF73AFB81
:105BA000FCF7ECF900BDEDE780CEFFF7B3FBFCF7A7
:105BB00003FC15206973206E6F7420696E205441B8
:105BC000534B20636861696E00BD0000AC0000208B
:105BD0000C530008C62E5441534B5320361F3760D8
:105BE000094F00B53F68002F0BD03D460C3D361FD6
:105BF00037602F46FBF704FAFCF70CFBFCF7BEF905
:105C0000F0E780CE00BD0000AC000020C0410008DD
:105C1000C82E52554E4E494E47202020361F376021
:105C2000064F00B5FCF798F9361F3760FFF7A6FF5F
:105C30003F6802488742F5D180CE00BD103F00206A
:105C40001176312E30205B6275696C642030303201
:105C5000375D14312041756720323032332C2031CA
:105C6000363A35373A33392000B5FCF775F9FCF789
:105C7000A3FB1C2A2A2A2A2A2A2A2A2A2A2A2A2A48
:105C80002A2A2A2A2A2A2A2A2A2A2A2A2A2A2A009E
:105C900000BD202000B5FFF7E7FFFCF75DF9FCF73A
:105CA0008BFB1C4D504520506F776572466F7274A8
:105CB0006820666F722053544D33324630373200BD
:105CC000FCF74AF9FCF778FB1C4D6F64696669655F
:105CD0006420666F722059656C6C6F77204D6F750C
:105CE0007365205632000000FCF736F9361F376026
:105CF000064FFCF72FFEFCF741F9361F3760044FC3
:105D0000FCF728FEFFF7B0FF00BD0000405C000874
:105D1000525C0008405A0008CA524550524F472E64
:105D2000494D472000B500BFFBF7C5FB305D0008BB
:105D3000FC0700204409002000000000006CDC0289
:105D400000000200000800003B1C83CE00D1704719
:105D5000021C0A431A430324144006D10A68026055
:105D6000091D001D1B1FF9D170470A780270491CDC
:105D7000401C5B1EF9D1704702CE0124E407734634
:105D80005B1E1A680919781A07B480CE7046001D88
:105D90000047000002CEB942EFD180CE012170460B
:105DA000884302681047361F37607046401E0768F8
:105DB00000BD000072B670473A4603CE0027121AA3
:105DC000091A914200D2FF437047000001CE3168AA
:105DD000202400224918404113465341C01B5B4117
:105DE00001D0491C00E0C019641EF3D10F46306099
:105DF00070472020361F0021316000B5FFF7E6FF15
:105E0000361D00BD0038014007480568002D03D04D
:105E10000548056805490D60044805680C202860A0
:105E20000D2028607047000008000020D4000020EA
:105E300007480568361F37602F4600BFFD69802080
:105E40000540FBD03068B8627768083670470000BC
:105E5000D400002004480568ED6920200540361F65
:105E600037602F4670470000D40000200A480568BC
:105E7000361F37602F4600BFFD6920200540FBD04C
:105E80007F6AFF20074000BF00BF00BF00BF00BF08
:105E900000BF00BF00BF7047D400002030683F182B
:105EA00030683760074600B5FFF774FF9D0100209A
:105EB000009D019805442D78361F37602F46FFF767
:105EC000B7FF0098401C0090F2D703B000BD20201F
:105ED000361F37600D2700B5FFF7AAFF361F376062
:105EE0000A27FFF7A5FF00BD07480568083E356093
:105EF0007760064F00B5FFF77DFF00BF7F1E002FC4
:105F0000FCD180CE00BD01BC0C00002020A1070008
:105F100007480568083E35607760064F00B5FFF713
:105F200069FF00BF7F1E002FFCD180CE00BD01BCE9
:105F30000C0000208813000000B500BFFFF7E8FF49
:105F40007F1E002FFAD180CE00BD202000B5FFF7C4
:105F500031FF054901200D6805430D6003480449E0
:105F6000086000BFFEE700BD24100240CCCC00005A
:105F70000030004000B500BFFFF715FF200A0020E9
:105F800000B500BFFFF70FFF240A002000B500BFD7
:105F9000FFF709FF280A002000B500BFFFF703FF45
:105FA0002C0A002000B500BFFFF7FDFE300A0020DC
:105FB00000B500BFFFF74EFF002F80CE03D0FFF7E4
:105FC00055FF80CEF6E700BD361F3760062700B5C7
:105FD000FFF72EFF00BD2020361F3760152700B5C4
:105FE000FFF726FF00BD2020361F3760182700B5B9
:105FF000FFF71EFF024901204042086000BD00007B
:10600000300A0020361F3760074F00B5FFF722FF28
:10601000002F80CE03D0FFF729FF361D00BD7F1E65
:10602000002FF3D1014F00BD00004000FFFFFFFF34
:10603000083E0021316077600C4F00B5FFF7E2FFAA
:1060400031680F7070683F18FF20074035686D1C7D
:1060500007488542EFF3008001B477602F46361D74
:1060600001BC80F30088E9D380CE00BD400A002047
:10607000C00A002000B5FFF7B7FFFFF7B5FF00BD6E
:1060800000B5FFF795FF07490868401C0860054800
:1060900005680548854202DDFFF7ECFF01E0FFF7E8
:1060A0009BFF00BD2C0A0020000100000748056886
:1060B000083E0749316077602F4600B500F0BCF913
:1060C000024908688030086000BD0000240A0020F2
:1060D000400A002000B5FFF795FFFFF793FF3068F7
:1060E0003F18FF2F80CE05D0FFF7CAFFFFF77CFFD8
:1060F00080CE00BD18480568FF200540BD4280CE17
:1061000002D0FFF7BDFF00BDFFF792FFFFF77AFF58
:1061100030688742EFF3008001B47768083601BC2D
:1061200080F3008802D0FFF7ABFF00BD0A48056886
:106130000A480468AC4202DAFFF79CFF00BDFFF793
:10614000B5FFFFF741FF04490868401C0860044997
:106150000020086000BD0000200A0020280A00205E
:106160002C0A0020361F37600A4F00B5FFF772FE79
:10617000002F01D0002701E001277F42306807404F
:1061800080CE03D0FFF7B0FE7F1EEFE780CEFFF793
:1061900061FE00BDA086010000B5FFF7E3FF002F00
:1061A00080CE03D1024901204042086000BD0000BA
:1061B000300A00202A49002008602A49002008608F
:1061C00000B5FFF7F5FEFF0927490F603068274942
:1061D00008600120264908601527361DFFF728FEB4
:1061E000FFF7C0FF002F80CE05D1361F376015277F
:1061F000FFF71EFEF4E700BFFFF7CEFF1848056863
:10620000002D1AD1FFF732FE042F06D104201449C5
:10621000086080CEFFF7D8FE0FE0182F06D11820B7
:106220000F49086080CEFFF7CFFE06E0012F03D1B3
:1062300080CEFFF74FFF00E080CE09480568002DB3
:10624000DAD007480568042DEFF3008001B4361F4B
:1062500037602F4601BC80F3008800D1002700BDC5
:10626000300A00202C0A0020280A0020240A0020DE
:10627000200A0020074805688020054000B508D0A6
:10628000054D06486860064868608020296981439A
:10629000296100BD10200240002002402301674513
:1062A000AB89EFCD083E134931607760124F00B5DE
:1062B0003068451E002DEFF3008001B4356001BC4D
:1062C00080F3008804D0FD6801200540002DEFD147
:1062D000FD6834242C40FC6030680028EFF3008017
:1062E00001B42F46361D01BC80F3008801D103485C
:1062F000074300BD000010000020024000000080A5
:1063000000B5FFF7B7FF084901200D6805430D6090
:106310003068388077680836FFF7C4FF02490120EB
:106320000D6885430D6000BD102002400B483F1AE8
:1063300000B5FFF79FFF0A4D02202969014329613B
:106340006F61402029690143296180CEFFF7AAFFD0
:10635000044902200D6885430D6000BD000000085F
:10636000002002401020024000B500BFFFF71BFDD7
:10637000340A0020202F80CE00B503D002490868DF
:10638000401C086000BD0000340A002030683F183F
:1063900030683760074600B5FFF7FCFC9306002025
:1063A000009D01980544361F37602F46FFF7BEFF5A
:1063B000FFF7E0FF03480568009840190090EFD709
:1063C00003B000BD1400002005480568083E0549DB
:1063D000316077602F4600B5FFF7D8FF00BD0000A1
:1063E00010000020000000087068054601218D4360
:1063F0003068044601218C437F1C01218F433F19E3
:1064000037607560274600B5FFF7C4FC050700201C
:106410003D88009C01980444083E3560776027461B
:10642000FFF76EFFFFF7A6FFBF1C0098801C0090CF
:10643000EED703B080CE00BD361F3760802700B591
:10644000FFF7D2FF00BD20200F200740092F00B525
:1064500000DDFF1D3037FFF7EBFC00BD3D0B361FA5
:1064600037602F4600B5FFF7EFFF3D0A361F376054
:106470002F46FFF7E9FF3D09361F37602F46FFF72C
:10648000E3FFFFF7E1FF00BD0845726173696E67C6
:10649000200620646F6E652010537461727420585A
:1064A0006D6F64656D20545820265072657373209B
:1064B0005220746F207265626F6F742C206F746845
:1064C000657220746F20726570726F6772616D20E3
:1064D000064572726F7273034E6F20207D1C3F78E9
:1064E000361F356000B5FFF7D9FC00BD00B5FFF7DA
:1064F000EFFC9C4D361F37602F46FFF7AFFF361F6E
:1065000037602027FFF794FC361F3760014FFFF7F5
:10651000E5FF00BDA007002000B5FFF775FC361FA2
:1065200037603227FFF708FD00BD202000B5FFF7D8
:10653000F3FF00BF284900200860FFF7C9FC361FA1
:106540003760264FFFF7CAFF361F37601427FFF763
:10655000F3FCFFF739FF361F3760214FFFF7BEFF0F
:10656000FFF7C4FF1C4900200860FFF7B1FC361F8D
:1065700037601C4FFFF7B2FF361F37601A27FFF74F
:1065800057FC19480568083E1849316077602F4666
:10659000FFF710FE80CEFFF7A9FF361F3760642794
:1065A000FFF7CAFCFFF794FC361F3760104FFFF768
:1065B00095FFFFF75BFCDF200740361F3760FFF7D2
:1065C00037FC522F80CEB5D1361F37606427FFF7D6
:1065D000B3FCFFF7BBFC00BD340A002058070020C5
:1065E000610700206807002010000020000000085C
:1065F0007907002005436F707920202000B5FFF750
:106600008BFFFFF765FC361F3760174FFFF766FFFC
:10661000361F37601427FFF78FFC144900200860ED
:10662000083EB16831607760FFF7B0FEFFF75EFFAC
:10663000361F37600A27FFF77FFC4A4D002D02D036
:10664000B7680C3600BDFFF743FC361F3760084FB4
:10665000FFF744FFFFF7C8FEFFF748FF361F37601C
:106660001427FFF769FC00BD58070020340A0020FA
:10667000C408002000B500BF0C3EF16831603169EC
:106680007160B760FFF7BAFF364D002DF4D1361FA9
:1066900037606427FFF750FCFFF758FC00BD00008F
:1066A000C8590008CB5245464C41534855415254B5
:1066B00000B500BFFAF732FFB0000020585B0008B9
:1066C000C643414C4C49542072B60F480568103EF1
:1066D0000E4931600E497160B560F7600D4F00B52D
:1066E000FAF748FB094DAF600B48E8600B4828619A
:1066F0000B48686135687768083601200543A8476C
:10670000FDF712F900BD0000B000002000000020DD
:10671000305D000870090000006CDC0200F8010028
:1067200000080000C0660008C75245464C41534867
:1067300004480568361F37602F4600B5FFF7C4FFD1
:1067400000BD0000305D0008185D0008C9434F50CF
:1067500059464C415348202004480568361F37608D
:106760002F4600B5FFF7B0FF00BD0000345D000804
:10677000EC5A0008CA4449534B2D4552524F5220FF
:1067800000B500BFFAF7CAFEB4000020A4660008F6
:10679000C8454E442D4C4F41442020205D460020EA
:1067A000E8625D46012040422863704700B500BFA3
:1067B000FBF794FB062F80CEFAD100BD361F376061
:1067C000002700B580CEFBF789FB152F01D00025EF
:1067D00001E001256D42062F01D0002701E00127CD
:1067E0007F422F43EFF3008001B42F4601BC80F3BA
:1067F0000088E7D000BD2020083E0021316077608E
:10680000064F00B5F9F78EFF306837600746FBF793
:1068100081FBFBF77FFBFFF7C9FF00BD0001000014
:1068200000B500BFFBF75AFB012F80CEFAD100BFA5
:10683000FBF762FB002F80CE03D0FBF74FFB80CE2F
:10684000F6E7361F37600627FBF764FB00BD202004
:1068500000B5FBF75FFBFFF7E3FF7D1C3F78083EC9
:1068600037607560FFF7C8FF361F3760002700BF2D
:10687000F9F734FE97680008009D01980544ED196A
:106880002D78361F37602F46FBF744FB0098401CDD
:106890000090F1D703B00627FBF73CFBFFF78EFF14
:1068A00001490F6080CE00BDB4000020361F376064
:1068B000052700B5FBF72EFBFBF74EFBFBF77CFD36
:1068C000084572726F72202320000000FBF78CFED7
:1068D000FBF754FBFBF77AFBFCF73CF8FBF73CFBC0
:1068E000FFF75CFF00BD2020361F3760062700B58C
:1068F000FFF7AEFF361F3760184FFFF77DFF361FDB
:1069000037600127FFF778FFFFF78AFF5D46002019
:1069100028635D4601204042E8620020104908607B
:10692000FCF77AFCFCF7B4F8361F37600D4FFBF725
:1069300053FD002F00D180CE0AD0FFF7B7FF5D4690
:10694000AD69361F37602F463E1C80CEFCF764FCD5
:106950005D462D6B002DE5D000BD01B4FFFFFFFFAC
:1069600098000020A0330008F4540008C7494E43A3
:106970004C554445361F3760202700B5FCF7FCF81E
:106980007D1C3C78083E356077602746FAF73CFA74
:10699000FFF7AAFF00BD000018580008C847454E81
:1069A000535049425220202030683760074600B5D6
:1069B000F9F756FF083E002131607760072700BFD6
:1069C000F9F78CFDEB690008009D0198054401244E
:1069D000AC40BC4204DA009F0198074403B000BDFC
:1069E0000098401E0090EFD703B0002700BD0000C4
:1069F00094590008C928494E495453504929202028
:106A000000B580B4009F402039688143396080CE52
:106A1000FFF7CAFFFF0007480743009D2F60009F54
:106A20000548786080BC402039680143396080CED9
:106A300000BD000007030000001700006C6900089B
:106A4000CD535049325F4E43535F4D454D53202047
:106A500000B500BFFAF72FFD5C6A00080008004887
:106A60000100000040000000285A0008C8535049A7
:106A7000325F53434B20202000B500BFFAF71BFDC7
:106A8000846A000800040048002000002D00000077
:106A90004C670008C9535049325F4D49534F20207D
:106AA00000B500BFFAF707FDAC6A00080004004813
:106AB000004000002E000000946A0008C9535049AD
:106AC000325F4D4F5349202000B500BFFAF7F3FC69
:106AD000D46A000800040048008000002F00000075
:106AE000F4690008C8495353504950494E202020AA
:106AF000083E00213160776000B5FDF779FE361F52
:106B000003213160FDF706FF00BD0000906700081B
:106B1000CA53454C494F2D5350493220174D184CFC
:106B2000696921436961A96AA143A962134D154CA2
:106B3000E9692143E9612969A1432961124D083EB0
:106B4000356077602F4600B5FDF742FE083E012113
:106B500031607760FDF7DEFEFDF758FD361F3760C8
:106B60000A4FFFF7C5FF361F3760094FFFF7C0FF19
:106B7000361F3760074FFFF7BBFF00BD0010024014
:106B80000000C000004000005C6A0008846A000841
:106B9000AC6A0008D46A000810520008C753504974
:106BA0005843484730683873361D00B5F9F7E8FC9C
:106BB000F9F7E6FCF9F7E4FCF9F7E2FCBD6883209D
:106BC0000540032DFAD13F7BFF20074000BD0000A8
:106BD0006C6A0008C8535049464C55534820202041
:106BE000361F3760044F00BFBD680120054001D04B
:106BF000FD68F9E780CE704700380040FC58000877
:106C0000C453504921202020361F3760024F00B561
:106C1000FFF7C8FF80CE00BD00380040006C0008C0
:106C2000C453504940202020083EFF213160776046
:106C3000024F00B5FFF7B6FF00BD0000003800406E
:106C4000E46A0008C8494E49545350493220202074
:106C500000B5FFF763FF0C3E0549316005497160DF
:106C6000B760054FFFF7CCFEFFF7BAFF00BD00008D
:106C7000006CDC0240420F0000380040745B0008EA
:106C8000C52E535049322020083E044931607760B8
:106C9000402700B5FEF7DEFB00BD000000380040D5
:106CA000D46B0008C853504944454C41592020201A
:106CB000361F3760092700BF7F1E002FFCD180CE12
:106CC00070470000BC6A0008C943534C4F5F4D45F4
:106CD0004D53202000B5FFF7EBFF361F3760034F01
:106CE000FDF7A0FCFFF7E4FF00BD00005C6A0008B0
:106CF000C86C0008C9435348495F4D454D53202097
:106D000000B5FFF7D5FF361F3760034FFDF77EFC58
:106D1000FFF7CEFF00BD00005C6A0008F46C0008BD
:106D2000C4484F4D45202020361F37601B2700B533
:106D3000FBF7F0F8361F37605B27FBF7EBF8361FE1
:106D400037604827FBF7E6F800BD000084580008CC
:106D5000C42E504F53202020361F37600A2700B51D
:106D6000F9F76EFD3037FBF7D5F83037FBF7D2F87F
:106D700000BD0000106B0008C6474F544F58592003
:106D8000361F37601B2700B5FBF7C4F8361F376086
:106D90005B27FBF7BFF8FFF7DFFF361F37603B27A6
:106DA000FBF7B8F8FFF7D8FF361F37604827FBF727
:106DB000B1F800BD74670008CB434C4541525343C2
:106DC0005245454E361F37601B2700B5FBF7A2F82A
:106DD000361F37605B27FBF79DF8361F3760322779
:106DE000FBF798F8361F37604A27FBF793F800BD8A
:106DF000786D0008CA5343524F4C4C444F574E20B5
:106E0000361F37601B2700B5FBF784F8361F376045
:106E10004427FBF77FF800BDA46C0008C853435219
:106E20004F4C4C5550202020361F37601B2700B593
:106E3000FBF770F8361F37604D27FBF76BF800BD86
:106E4000206D0008C95343524F4C4C494E472020F7
:106E5000361F37601B2700B5FBF75CF8361F37601D
:106E60005B27FBF757F8361F37607227FBF752F89E
:106E700000BD0000446E0008C9435552534F524FA5
:106E800046462020361F37601B2700B5FBF742F827
:106E9000361F37605B27FBF73DF8361F37603F270B
:106EA000FBF738F8361F37603227FBF733F8361F09
:106EB00037603527FBF72EF8361F37606C27FBF756
:106EC00029F800BD1C6E0008C8435552534F524F5D
:106ED0004E202020361F37601B2700B5FBF71AF81D
:106EE000361F37605B27FBF715F8361F37603F27E3
:106EF000FBF710F8361F37603227FBF70BF8361F09
:106F000037603527FBF706F8361F37606827FBF731
:106F100001F800BD085B0008C345534300B500BF3E
:106F2000FAF7C9FA1B000000406A0008C43C23239A
:106F30003E2020205D46AD6B00B520B4FBF7BAFAC9
:106F4000361F37600027FBF7FDFAFBF7EDFAFBF77A
:106F500003FBFAF7F1FF20BC5C46A56300BD00000F
:106F600028670008C44553435B202020361F376044
:106F70001B2700B5FAF7CEFFFBF71EFA015B0000F6
:106F800000BD0000C86E0008C744454641554C543A
:106F900000B500BFFAF78FFA00000000105C00088F
:106FA000C4424F4C4420202000B500BFFAF783FABA
:106FB00001000000206C0008C344494D00B500BF2B
:106FC000FAF779FA020000009C690008C6495441AA
:106FD0004C49432000B500BFFAF76DFA03000000EA
:106FE000B86D0008C9554E4445524C494E452020C5
:106FF00000B500BFFAF75FFA04000000B86F0008A0
:10700000C5424C494E4B202000B500BFFAF753FA59
:107010000500000048550008C352455600B500BFA2
:10702000FAF749FA0700000000700008C5424C4119
:107030004E4B202000B500BFFAF73DFA08000000D3
:107040002C700008C5424C41434B202000B500BFC6
:10705000FAF731FA0000000018700008C3524544E6
:1070600000B500BFFAF727FA01000000786E0008AB
:10707000C5475245454E202000B500BFFAF71BFA20
:1070800002000000CC6F0008C659454C4C4F5720F9
:1070900000B500BFFAF70FFA03000000A06F000868
:1070A000C4424C554520202000B500BFFAF703FA32
:1070B00004000000D45B0008C74D4147454E5441D1
:1070C00000B500BFFAF7F7F90500000044700008AA
:1070D000C44359414E20202000B500BFFAF7EBF918
:1070E0000600000070700008C5574849544520202C
:1070F00000B500BFFAF7DFF9070000005C70000878
:10710000C44154545220202000B5FFF72FFFFFF751
:1071100011FFFBF751F9016D00BD0000186F000869
:10712000C4544558542020201E3700B5FFF7ECFF0B
:1071300000BD0000E8700008CA4241434B47524F6F
:10714000554E4420283700B5FFF7DEFF00BD000094
:10715000D0700008C552464C4544202000B500BF01
:10716000FAF7A9F96871000800080048002000003B
:107170004D0000002C6F0008C44C4F444F202020CD
:1071800000B500BFFAF797F98C71000800000048BD
:1071900002000000010000009C6B0008C85246532A
:1071A00049474E414C20202000B500BFFAF783F933
:1071B000B47100080000004808000000030000004F
:1071C0009C710008C852575349474E414C2020201B
:1071D00000B500BFFAF76FF9DC7100080000004845
:1071E0001000000004000000B8700008C84C4653AE
:1071F00049474E414C20202000B500BFFAF75BF90B
:107200000472000800000048200000000500000093
:10721000EC710008C84C575349474E414C20202080
:1072200000B500BFFAF747F92C72000800000048CB
:107230004000000006000000446C0008C54C464CAD
:107240004544202000B500BFFAF735F95072000818
:107250000000004880000000070000003C720008A9
:10726000C54C574C4544202000B500BFFAF723F920
:1072700074720008000400480100000020000000B3
:10728000A0700008C353573100B500BFFAF713F9D7
:107290009472000800040048020000002100000071
:1072A00084720008C353573200B500BFFAF703F9E0
:1072B000B47200080004004804000000220000002E
:1072C000E46F0008C6284C50574D292000B500BF78
:1072D000FAF7F1F8D8720008000000480001000039
:1072E00008000000C4720008C6285250574D2920DB
:1072F00000B500BFFAF7DFF8FC7200080000004894
:10730000000800000B000000646F0008C950574DD2
:10731000454E41424C45202000B500BFFAF7CBF85E
:107320002473000800000048001000000C0000005A
:10733000806C0008C74C4D41524B455200B500BF10
:10734000FAF7B9F848730008000000480040000050
:107350000E0000000C730008C7524D41524B4552BD
:1073600000B500BFFAF7A7F86C73000800000048EA
:10737000008000000F000000A4720008C4524F44B7
:107380004F20202000B500BFFAF795F89073000851
:10739000000400481000000024000000887000086D
:1073A000C8475245454E4C454420202000B500BFFB
:1073B000FAF781F8B87300080004004820000000C4
:1073C00025000000506D0008C959454C4C4F574CE2
:1073D0004544202000B500BFFAF76DF8E0730008BF
:1073E0000004004840000000260000002071000852
:1073F000C65245444C45442000B500BFFAF75BF83F
:107400000474000800040048800000002700000009
:10741000F0730008C5534F554E44202000B500BFFF
:10742000FAF749F828740008000400480001000039
:107430002800000054710008C552574C45442020D4
:1074400000B500BFFAF737F84C7400080004004894
:107450000002000029000000C8730008C9492F4F2E
:10746000434C4F434B5320200F4D10486969014353
:1074700069610F48A9690143A9610320E9690143D2
:10748000E9612C460C340A4B2168194321602168BC
:10749000994321602C46103403232168194321604D
:1074A00021689943216070470010024001000E00DE
:1074B000000A060014720008C450574D4C202020CA
:1074C00001490F6080CE7047342C0140B874000829
:1074D000C450574D5220202001490F6080CE704784
:1074E000402C0140D0740008C84C45465453544FBA
:1074F0005020202000B500BFF9F7DDFFD4010000C7
:10750000886F0008C9524947485453544F502020AF
:1075100000B500BFF9F7CFFFD4010000F46D0008FB
:10752000CA53544F504D4F544F525320361F37605B
:10753000044F00B5FFF7C4FF361F3760014FFFF758
:10754000CBFF00BDD4010000A0730008C6494E491E
:107550005454312000B5FFF7E9FF0F4D0F48E862A2
:107560006020A8610E48E8610E4828620020A862E9
:107570000D48686401202860083E02213160776070
:107580000A4FFDF735F9083E022131607760084F58
:10759000FDF72EF900BD0000002C0140E8030000BB
:1075A000006000000110000000800000D872000898
:1075B000FC72000834730008C74C504552494F44D0
:1075C00002480588361F37602F4670473800004054
:1075D00058730008C752504552494F440248058825
:1075E000361F37602F46704734040040B8750008D6
:1075F000CA494E4954504552494F44200448F86204
:107600002F20B862012038603120386280CE704768
:10761000FFFFFFFF60720008C8494E495454322FE3
:1076200033202020134D1448E8601448A860144803
:10763000A861361F37602F4600B5FFF7DFFF114DF9
:107640001148E8601148A8601148A861361F3760EA
:107650002F46FFF7D3FF083E0221316077600D4FC0
:10766000FDF7C6F8083E0121316077600A4FFDF74B
:10767000BFF800BD000000400004000064010000ED
:10768000111100000004004000020000540100003D
:10769000111000008C710008907300085C740008E1
:1076A000C64C434F554E54200348056803494D1BB3
:1076B000361F37602F46704734000240FFFF00003E
:1076C00038740008CB4C434F554E54434C454152FF
:1076D000044D0020286004480449086031202860D7
:1076E0007047000030000240FFFF000034000240FD
:1076F00014740008C652434F554E54200348056881
:1077000003494D1B361F37602F4670474800024023
:10771000FFFF000020750008CB52434F554E5443E5
:107720004C454152044D002028600448044908603B
:10773000312028607047000044000240FFFF000035
:107740004800024038710008C8444D41494E495430
:1077500033202020044D0548A8630548E86300B5A0
:10776000FFF7B6FF00BD00000000024024480140C2
:107770000000000848770008C8444D41494E49546C
:1077800034202020044D0548E8640548286500B5EC
:10779000FFF7C8FF00BD0000000002402448014080
:1077A00000000008E8720008CB434C454152434FAB
:1077B000554E545300B5FFF78BFFFFF7B3FF00BDE5
:1077C00078770008CA5246414E414C4F47554520F4
:1077D00000B500BFF9F76FFE08000000187600083A
:1077E000C54C494E4530202000B500BFF9F763FE77
:1077F00008000000C4770008CA5257414E414C4F60
:107800004755452000B500BFF9F755FE10000000B0
:10781000E0770008C54C494E4531202000B500BF37
:10782000F9F749FE100000007C730008CA4C46417D
:107830004E414C4F4755452000B500BFF9F73BFE80
:107840002000000014780008C54C494E4532202025
:1078500000B500BFF9F72FFE200000002C780008CB
:10786000CA4C57414E414C4F4755452000B500BFCB
:10787000F9F721FE4000000048780008C54C494E49
:107880004533202000B500BFF9F715FE4000000089
:10789000F4760008C7414E414C4F4753361F3760BE
:1078A000094F00B5FCF7C6FF361F3760074FFCF7DE
:1078B000C1FF361F3760064FFCF7BCFF361F37602D
:1078C000044FFCF7B7FF00BDB4710008DC7100087D
:1078D000047200082C720008C4760008C6414443B4
:1078E0005F43522000B500BFF9F7E5FD08240140D1
:1078F000E8740008C341444300B500BFF9F7DBFD5D
:1079000000240140D4750008C8414443444F4E450B
:107910003F2020200648056804200540002D01D0A6
:10792000002501E001256D42361F37602F46704764
:1079300008240140A0760008CB57414954414443F4
:10794000444F4E4500B500BFFFF7E4FF002F80CE47
:10795000FAD000BD38790008CB5741495443414C17
:10796000444F4E4500B500BF02480568002DFBD1CD
:1079700000BD01B408240140F8770008CB4144431E
:10798000454E41424C45443F0348056801200540AF
:10799000361F37602F46704708240140947800084E
:1079A000C74144435F43414C00B5FFF7EDFF002F53
:1079B00080CE02D0022006490860FFF7D3FF0020E6
:1079C00003490860034802490860FFF7CBFF00BD88
:1079D0000824014000000080C4710008C9414443EC
:1079E000454E41424C45202000B5FFF7DDFF012008
:1079F0000149086000BD00000824014078710008BA
:107A0000C9574149545245414459202000B500BF4F
:107A10000248056801200540FAD000BD002401405D
:107A200008790008C841444353544152542020204F
:107A3000024904200D6805430D6070470824014089
:107A4000007A0008C7494E495441444300B5FFF746
:107A500025FFFFF7A9FFFFF7C7FFFFF7D7FF044D8B
:107A60000020E860034828610420686100BD000030
:107A70000024014000000080A0790008C54348535D
:107A8000454C202000B500BFF9F715FD2824014022
:107A90007C7A0008C74144434441544100B500BFCB
:107AA000F9F709FD4024014000710008C441544F1A
:107AB0004420202006490F6080CE00B5FFF7B8FFB4
:107AC000FFF740FF03480568361F37602F4600BDAB
:107AD000282401404024014004750008C754494D42
:107AE0004552313600B500BFF9F7E5FC00440140CE
:107AF000A8770008CB534F554E44504552494F4448
:107B000001490F6080CE70472C440140DC790008A9
:107B1000C7534F554E444F4E012005490860083E5B
:107B2000022131607760034F00B5FCF761FE00BDB4
:107B30000044014028740008DC7A0008C8534F55FF
:107B40004E444F4646202020002007490860361F3B
:107B50003760064F00B5FCF73BFE361F3760034F1A
:107B6000FCF760FD00BD00000044014028740008DF
:107B7000447A0008C7494E4954543136064D3020E6
:107B8000A86101202862054868641720A86200B532
:107B9000FFF7DAFF00BD0000004401400080000054
:107BA00058790008C9494E49545354554646202037
:107BB00000B5FFF759FCFFF735FDFFF7CBFDFFF7E9
:107BC000E1FDFFF7C7FCFFF7D9FFFFF73FFF00BD5F
:107BD000F0750008CA494E4954414C4C492F4F207A
:107BE00000B5FFF7E5FF2E4D083E356077602F4664
:107BF000FCF7EEFDFCF716FD2A4D083E3560776078
:107C00002F46FCF7E5FDFCF70DFD274D083E3560DE
:107C100077602F46FCF7DCFDFCF704FD234D083EA2
:107C2000356077602F46FCF7D3FDFCF7FBFC204D59
:107C3000083E356077602F46FCF7CAFDFCF7F2FC82
:107C40001C4D083E356077602F46FCF7C1FDFCF700
:107C5000E9FC194D083E356077602F46FCF7B8FD0A
:107C6000FCF7E0FC154D083E356077602F46FCF7C9
:107C7000AFFDFCF7D7FC361F3760114FFCF798FDBE
:107C8000361F37600F4FFCF793FD361F37600E4FDE
:107C9000FCF78EFD361F37600C4FFCF789FD00BDE9
:107CA000687100084C740008507200087472000873
:107CB00004740008E0730008B87300082473000817
:107CC0006C7300084873000894720008B4720008CE
:107CD00000000000E07B0008DC780008C453573146
:107CE0003F202020361F3760054F00B5FCF7A6FC6B
:107CF000002F01D0002701E001277F4200BD0000D6
:107D000094720008DC7C0008C45357323F202020C6
:107D1000361F3760054F00B5FCF790FC002F01D0EF
:107D2000002701E001277F4200BD0000B472000877
:107D3000947A0008C652502D454E442000B500BF2D
:107D4000F9F7B9FB4C36002018770008CA534554A0
:107D5000434F4E534F4C45205D46EF645D46AF6444
:107D600080CE7047107B0008C54552415345202006
:107D7000361F3760002700B5F9F7A2F800BD0000F4
:107D8000B80000000000002000000000000000001B
:107D9000000000008005000800000000E80000006E
:107DA00000000000000000000000000000000000D3
:107DB000000000001800002000000000000000008B
:107DC0000000000000000000000000008005000826
:107DD00000000000981E000810000000747B0008DE
:107DE0007C780008A47B0008D47B0008F4780008A5
:107DF000AC7A000860780008087D0008347D00082F
:107E0000247A0008687D00083C7B00087C79000823
:107E10004C7D0008F47A00084C7500080000000052
:107E20004028000800000000D07C0008010000008D
:107E30000000000000000000105800080038014059
:107E40000000000000000000000000000000000032
:00000001FF
